:105AE100755606123C11202B04E54470F9123C5AFC
:105AF100755606123BD180E822755604123C11E519
:105B01004470FC123C5A755604123BD17F01123687
:105B1100707E007FFF8F0512585CDFF97E007FFFEA
:105B2100900000C007125899EFF0A3D007DFF422CC
:105B3100755601123C11E54470C5123C5A75560167
:105B4100123BD12275570112367078083029FDE5D4
:0B5B5100492430123641C229D8EA2254
:102C0B007584008537D28538D37584018539D28593
:102C1B003AD3E4F538F537300006853B37853C3839
:102C2B0030010CE537253DF537E538353EF53830C5
:102C3B000210E548852EF0A42537F537E5F0353839
:102C4B00F538300310E50A8531F0A42537F537E563
:102C5B00F03538F538300410E5118530F0A4253700
:102C6B00F537E5F03538F538E4F53AF53930081035
:102C7B00853B39853C3AE53CC39535400385353A70
:102C8B00300916E53EC39534400385353EE53925BD
:102C9B003DF539E53A353EF53A300A10E548852ED3
:102CAB00F0A42539F539E5F0353AF53A300B10E556
:102CBB000A8531F0A42539F539E5F0353AF53A3086
:102CCB000C10E5118530F0A42539F539E5F0353ACE
:102CDB00F53A300D10E518852FF0A42539F539E5B7
:102CEB00F0353AF53A300E10E52C8533F0A4253942
:102CFB00F539E5F0353AF53A300F10E52D8532F020
:102D0B00A42539F539E5F0353AF53AE53AC3953668
:102D1B00400385363A22902E10302D03122D45306C
:072D2B002E03122D5530307C
:102D320003122DBD302F05B2A1122D7830310312AE
:102D42002DCD22E50B2509F50BE50C3508F50C9385
:102D5200F50A22E512250EF512E513350DF513934A
:102D6200C313F8E5142510F514E515350FF5159381
:102D7200C31328F51122B2A0103908203A3C303D85
:102D8200238026D23A203B0E303C2FC23AC23DD29B
:102D92003B756C008024203C21C23AD23DC23B7577
:102DA2006C008016902F108003902F58E56C93F5DD
:102DB2002C056CE56CB44802D23A22E5192517F5C8
:102DC20019E51A3516F51A93F51822103E08203F18
:102DD2003C3042238026D23F20400E30412FC23F5A
:102DE200C242D240756D008024204121C23FD242AE
:102DF200C240756D008016902FC08003902FA0E511
:102E02006D93F52D056DE56DB44802D23F227F82A8
:102E120085888C8F9295989B9EA1A4A7AAADB0B3EA
:102E2200B6B9BBBEC1C3C6C9CBCED0D3D5D7D9DC08
:102E3200DEE0E2E4E6E7E9EBEDEEF0F1F2F4F5F6DE
:102E4200F7F8F9FAFBFCFCFDFDFEFEFEFEFEFEFEBF
:102E5200FEFEFEFDFDFCFCFBFAFAF9F8F7F6F4F3D0
:102E6200F2F0EFEDECEAE8E7E5E3E1DFDDDBD8D60F
:102E7200D4D1CFCDCAC8C5C2C0BDBAB7B4B2AFAC47
:102E8200A9A6A3A09D9A9794908D8A8784817E7A21
:102E92007774716E6B6865625F5C595653504D4A28
:102EA2004744423F3C393734322F2D2A28262421E9
:102EB2001F1D1B1918161412110F0E0C0B0A0807EE
:102EC20006050404030202010100000000000000E4
:102ED20000000001010202030405060708090A0BAB
:102EE2000D0E1011131516181A1C1E202224272944
:102EF2002B2E303335383A3D404245484B4E5154E3
:102F020056595C606366696C6F7275787B7FFEFEF2
:102F1200FEFEFDFCFCFBFAF8F7F6F4F3F1EFEDEB45
:102F2200E9E7E4E2DFDCDAD7D4D0CDCAC6C3BFBC5E
:102F3200B8B4B0ACA8A39F9B96928D89847F7A7512
:102F4200706B66615C57514C47413C37312C2621EE
:102F52001B16100B050000050B10161C21272C3226
:102F6200373D42484D53585D62686D72777C81856A
:102F72008A8F94989DA1A5AAAEB2B6BABEC1C5C8A1
:102F8200CCCFD2D5D8DBDEE1E3E6E8EBEDEFF1F230
:102F9200F4F6F7F8F9FBFBFCFDFEFEFEFEFE000C6C
:102FA2001926333F4C5864707B86919CA6AFB8C1FA
:102FB200C9D1D8DEE4EAEFF3F6F9FCFDFEFEFEFD30
:102FC200FCFAF7F4F0EBE6E0DAD4CCC5BCB4ABA182
:0E2FD200978D83786D61554A3D3125180C00AE
:10359E00D2F4C2F5C2F675840F85F0C81233CE741C
:1035AE00031235ED1233C274031235ED1233A51228
:1035BE0033A574031235ED1233A574021235ED12D4
:1035CE0033A574281236597406123659740E1236F3
:1035DE005974011236591233C2748012365922C0F0
:1035EE0000A2E092F3A2E192F2A2E292F1A2E392A1
:1035FE00F0D2F475840F85F0C8C2F47830D8FE8509
:10360E00F0C87830D8FED00022C00075840FA2E436
:10361E0092F3A2E592F2A2E692F1A2E792F0D2F430
:10362E0085F0C8C2F47830D8FE85F0C87830D8FE60
:10363E00D00022EF75840FD2F5C2F685F0C812368F
:10364E00171233A51235ED1233A52275840FC2F56C
:10365E00C2F685F0C81236171233A51235ED1233A5
:10366E00A522EF14A2E492E6C2E4D2E71236592262
:10367E00740F12365922740D123659227F011236EA
:10368E007078107F20123641D8F9227F11123670D1
:10369E0078107F20123641D8F9227F0112367078C9
:1036AE00207F20123641D8F922C0077F018004C046
:1036BE00077F11123670D007C082C083C007EF7526
:1036CE00F0109036E81233E67810E493FF1236418C
:0936DE00A3D8F7D007D083D082F5
:1036E70022202020202020202020202020202020D1
:1036F7002030313233343536373839414243444547
:10370700462020205253343232205445535420202F
:103717002020202052533233322054455354202046
:103727002020205445535420204641494C454420ED
:1037370020202054455354202050415353454420C2
:10374700202020454550524F4D20544553542020AA
:1037570020204155582052454C4159205445535437
:103767002020205055534820544F2054414C4B2083
:103777002054455354203320434841522F53554238
:1037870020544553542046495845442053545249E0
:103797004E5445535420564152494220535452499E
:1037A7004E464143544F52592044454641554C5487
:1037B7002050524F4752414D4D494E47204D4F449F
:1037C7004553494D504C4558205245504541544565
:1037D700522020205245434F5244494E4720202033
:0137E70020C1
:10585C00758400D2C2C2C6D2C6C2C4D2C5C2C330BD
:10586C00C3FD74A0F5C2C2C5C2C330C3FD8EC2C293
:10587C00C330C3FD8FC2C2C330C3FD8DC2C2C3309F
:10588C00C3FDD2C4C2C320C4FD1233C2227584002E
:10589C00C2C3D2C530C3FD74A0F5C2C2C5C2C330E9
:1058AC00C3FD8EC2C2C330C3FD8FC2C2C330C3FDA1
:1058BC00C2C4D2C5C2C330C3FD74A1F5C2C2C5C235
:1058CC00C330C3FDC2C2C2C330C3FD85C207D2C43C
:0658DC00C2C320C4FD223E
:080003000239DF0000000000DB
:08000B000239E30000000000CF
:08001300023B3E00000000006A
:08001B003200000000000000AB
:09002300320000000000000000A2
:08002B000239E60000000000AC
:08003300320000000000000093
:0A003B003200000000000000000089
:0900430032000000000000000082
:08004B0032000000000000007B
:08005300320000000000000073
:08005B00023A4B000000000016
:08006300320000000000000063
:08006B00023A630000000000EE
:080073000239EC00000000005E
:08007B00023B410000000000FF
:08008300023A450000000000F4
:08008B0032000000000000003B
:10009300023B5F00000000000000000000000000C1
:1000A3003275FF0775FFDE75FFAD75840F75E107C8
:1000B30075E20475E34475840F75A43575A5097558
:1000C300A6FF75A7FF759CFF759D00759E00759F24
:1000D300F075D8FF75E8FF75F80F75AD0F758401DE
:1000E30075893075888F75840275893075888F7529
:1000F300840F758A80758C67780874FF0000000090
:100103000000000000000000D5E0F1D8EDE58C30E0
:10011300E7FB759701758A0043890475840075B7F9
:100123001075840F438901758D01758F01758E02DA
:100133007480D5E0FD438902E58930E4FB759702BD
:1001430075840075D10775840075BB0175BA007598
:10015300BCF075C70075C60075C5FF75C4FF75E8AB
:100163008175840275BB0475BA0075BCF175C60050
:1001730075C4FF75E88875840075D484758401752A
:10018300D484758400C2F8759A47759D1A43F8099B
:1001930075870075840075B90075A90075910075A0
:1001A300985075840175981075840075C04075C3A7
:1001B3000075CFC9758400758E0075892075880513
:1001C300758400758A00758B6F758CF4758D6F431C
:1001D300885075840075C90075CA0075CB0075CC4D
:1001E3000075CD0075840175C91875CA8075CBFB80
:1001F30075CDFB75CC80D2CA75840275C91875CAD2
:10020300A675CBAF75CDAF75CCA6D2CA7584007574
:10021300EF0075A8AF75B80075E6A475E71775F616
:100223000075F7019000007F007E20E4F0A3DFFC5F
:02023300DEFAF1
:10023500752EFF752FFF7530FF7531FF7532FF7510
:0C02450033FF7534FF7535FF7536FF225E
:1039DF00022FE032C28D32758400C2CF32C0E0C0F8
:1039EF0083C082C0D0C000C0F0C2CFB23220322319
:1039FF00122C0B151BE51B7009751B0A75840175BD
:103A0F0088AF151CE51C7009751C607584027588DC
:103A1F00AF8011122D21153FE53F7008753F0475DA
:103A2F008400D28B758400D2ECD0F0D000D0D0D0EF
:103A3F0082D083D0E032C2CF0210AF32C0E0C0D00C
:103A4F00E54060021540E5436002154375888FD04D
:103A5F00D0D0E032C0E0C0D0C000C084202A13759F
:103A6F00840F30DF25E5E8540FF549D22A754AC88F
:103A7F008018154AE54A7006E549D2E7F54975847D
:103A8F000F20DF06C22AD229D251202C1475840FA1
:103A9F0030F828E5E854F0C4F54BD22C754CC880AB
:103AAF001A154CE54C7006E54BD2E7F54B75840FB4
:103ABF0020F808C22CD22BD250D237E54160021524
:103ACF0041E55E6002155E787FE6600116151DE523
:103ADF001D7051751D0AE54260021542E5446002F2
:103AEF001544E55A6002155AE55B6002155B788B49
:103AFF00E6600116E55860021558E5596002155940
:0D3B0F00151EE51E701E751E0AE55D6002A4
:103B1C00155DE57860021578151FE51F7009751F96
:103B2C0006E55C6002155CD084C28DD000D0D0D08C
:103B3C00E032020DB720280DD22885BF3E85BE3D50
:103B4C0075BB01800BC22885BF3C85BE3B75BB0095
:103B5C00C2ED32C0E0C0D0E54DB4000A054D85BEC3
:103B6C004875BB07803DB4010A054D85BE4575BB44
:103B7C00048030B4020A054D85BE4875BB0680230F
:103B8C00B4030A054D85BE4675BB048016B4040A01
:103B9C00054D85BE4875BB058009754D0085BE4732
:0A3BAC0075BB04C2EDD0D0D0E032AA
:1033350075840FD2FD2275840FC2FD2275840FD2CC
:10334500FC2275840FC2FC2275840FD2FED2452261
:1033550075840FC245C2FE22C29322D29322758480
:103365000FA2FA2275840FA2F92275840FA2DD221D
:1033750075840FA2DE22A2922275840FA2DA22752D
:10338500840FA2DB2275840FA2D82275840FA2D9DF
:1033950022000000000000000000000000000022E4
:1033A500C000C001790478B4D8FED9FAD001D000A4
:1033B50022C00078141233A5D8FBD00022C0E075D6
:1033C5004005E54070FCD0E022C0E075400FE540C7
:1033D50070FCD0E022C0E0754064E54070FCD0E0B0
:1033E50022A42582F582E58335F0F58322B40A000F
:1033F50022C0E0C3997001D3D0E022B50601225066
:1034050007B5070122400122D322EF75F064842419
:10341500309000A1F0E5F0A375F00A842430F0A304
:10342500E5F02430F022EF75F0648424309000A19B
:07343500F0E5F0A375F00AB9
:10343C00842430F0A3E5F02430F09000A1E0B43007
:10344C000B7420F0A3E0B430037420F02290000D34
:10345C00E0540FFFA3E0B420028019540FCF75F095
:10346C000AA42FFFA3E0B420028009540FCF75F0FB
:10347C000AA42FFF22C006C005C00490000DE05422
:10348C000FFFFEA3E0B42003C3802C540FFDCF75B7
:10349C00F00AA42FFFA3E0B42003C3801A540FFC3E
:1034AC00EE75F064A420D20EFEED75F00AA42E4049
:1034BC00052C40028001D3D004D005D0062275F033
:1034CC006484F6E5F00875F00A84F608A6F0082284
:1034DC00C0017900E6B4FF028027F908E6B4FF03C7
:1034EC00C38022E975F00AA426F908E6B4FF03C3E9
:1034FC008013E975F00AA420D207C3264003F98093
:10350C0004D3D00122E9D00122E675F00AA40826E2
:10351C00227850EE1234CA754E00754F00785290D6
:04352C00357679086F
:10353000EF134007A3A3A3A3A3801CC0E0C000C057
:1035400001C37905E49336D4A2E4540FF6A318D945
:10355000F3D001D000D0E0D9D8E54E600C754F090A
:10356000755009755109755209854F4E85504F8523
:10357000515085525122060502000002010500004B
:103580000402000100080400020006090004000211
:0E3590000901080004080306010806070203EB
:1022F00044313233343536373839302A234142437A
:1023000044AAA3C1C2C3C4D7ABA8A92A234142434C
:1023100001010101010101010100000000000000B4
:1023200000000000000000000000000000000000AD
:10233000000000000000000000000000000000009D
:10234000000000000000000000000000000000008D
:10235000000000000000000000000000000000007D
:102360000000000000000000000001010101010167
:10237000010101000000000000000000000000005A
:10238000000000000000000000000000000000004D
:10239000000000000000000000000000000000003D
:1023A000000000000000000000000000000000002D
:1023B000000000000000000000000000000000001D
:1023C0000000000001010101010101010100000004
:1023D00000000000000000000000000000000000FD
:1023E00000000000000000000000000000000000ED
:1023F00000000000000000000000000000000000DD
:1024000000000000000000000000000000000000CC
:1024100000000000000000000000000000006E0648
:10242000001102061501016E1006110301150101CC
:1024300064011611040515010100000000000000F0
:10244000000000000000000000000000000000008C
:10245000000000000000000000000000000000007C
:10246000000000000000000000000000000000006C
:102470000000000000000000010101010101010154
:10248000010000000000000000000000000000004B
:10249000000000000000000000000000000000003C
:1024A000000000000000000000000000000000002C
:1024B000000000000000000000000000000000001C
:1024C000000000000000000000000000000000000C
:1024D00000000101010101010101010000000000F3
:1024E00000000000000000000000000000000000EC
:1024F00000000000000000000000000000000000DC
:1025000000000000000000000000000000000000CB
:1025100000000000000000000000000000000000BB
:10252000000000000000000000000000202020202B
:10253000202020202020202020202020202020209B
:10254000202020202020202020202020202020208B
:10255000202020202020202020202020202020207B
:10256000202020202020202020202020202020206B
:10257000202020202020202020202020202020205B
:10258000202020202020202020202020202020204B
:10259000202020202020202020202020202020203B
:1025A000202020202020202020202020202020202B
:1025B000202020202020202020202020202020201B
:1025C00020202020202020202020202020202041EA
:1025D0004E49204E554D424552202020202020209B
:1025E000414E49204E414D45202020202041555844
:1025F0002052454C41592056414C4944202020202E
:102600002020202020202020313D454E2020202049
:10261000202020202020202020414E492020202042
:1026200020202020202020202020202020202020AA
:10263000202020202020202020202020202020209A
:10264000474C4F42414C202020202020204354431F
:10265000535320434F444520202020202020444332
:102660005320434F44452020202020204C5452200A
:1026700052455045415445522020202020414E498A
:1026800020504152414D45544552532053504545E9
:10269000442043414C4C494E472020202050544375
:1026A000204E554D424552202020202020564F4993
:1026B0004345204D455353414745532020564F49EC
:1026C000434520504C41594241434B202020494E24
:1026D00056414C49442054595045202020204F5504
:1026E00054204F462052414E4745202020494C4C13
:1026F0004547414C2056414C554520204D5553549B
:102700002046494C4C204649454C44202020494C09
:102710004C4547414C20434F4445202020444154E0
:102720004120414343455054454420204C494E45A7
:10273000204E554D4245523A2020202055534552B7
:102740002050524F4752414D4D494E4755534552E7
:102750002049443A2020202020202020564F494361
:1027600045205245434F5244494E472020494C4C46
:102770004547414C20454E545259202020494C4C4D
:102780004547414C2047414E4720202020202043F0
:102790004F4D504C45544544202020203633303690
:1027A00037303639343731393734343737303739D1
:1027B00037383235383534383835393135393438B9
:1027C00039373431303031303331303731313031E5
:1027D00031343131383132333132373133313133D1
:1027E00036313431313436313531313536313539B0
:1027F00031363231363531363731373131373331A1
:102800003737313739313833313836313839313972
:102810003231393631393932303332303632313083
:102820003231383232353232393233333234313276
:102830003530323534303036303037303135303174
:102840003730323130323330323530323630333166
:102850003033323033363034333034373035303053
:102860003531303533303534303635303731303737
:10287000323037333037343131343131353131362C
:102880003132323132353133313133323133343127
:102890003431313433313435313532313535313508
:1028A00036313632313635313732313734323035F0
:1028B00032313232313432323332323532323632F0
:1028C00034333234343234353234363235313235D1
:1028D00032323535323631323633323635323636BB
:1028E00032373132373433303633313133313533B7
:1028F00032353333313333323334333334363335A3
:10290000313335363336343336353337313431318C
:10291000343132343133343233343331343332348A
:102920003435343436343532343534343535343660
:102930003234363434363534363635303335303655
:102940003531363532333532363533323534363546
:102950003635363036363132363234363237363333
:102960003136333236353436363236363437303324
:102970003731323732333733313733323733343715
:1029800034333735344142434445464748494A4B3E
:102990004C4D4E4F505152535455565758595A61F9
:1029A00062636465666768696A6B6C6D6E6F70718F
:1029B00072737475767778797A303132333435368C
:1029C000373839607E21402324255E262A28295F56
:1029D0002D2B3D7B7D5B5D7C3A3B3C3E2C2E3F2F7F
:1029E0002020202020202020206401001102111529
:1029F00001016402001103111501016404001104B6
:102A00001115010164080011051115010178060175
:102A100011060119010182020711071215006382D4
:102A2000020811081215006382020911091315002A
:102A30006382030A110A151500FF82030B110B159F
:102A40001500FF641000110C1115051982020C11FC
:102A50000D1415016382020D110E1415006382021C
:102A60000E110F1415006382020F1110131501636C
:102A70002020202020202020202020202020202056
:102A80002020202020202020202020202020202046
:102A90002054454C434F2050524F4752414D202027
:102AA00020524144494F2050524F4752414D20201F
:102AB0002050484F4E452050524F4752414D202004
:102AC00020434F4D50552050524F4752414D2020EA
:102AD000202041434345535320434F444520202069
:102AE000205455524E204F4E2044454C41592020F1
:102AF000205455524E204F46462044454C415920C3
:102B00005455524E2041524F554E4420444C59206A
:102B100044544D462054454C434F204C4556454C5B
:102B200044544D4620524144494F204C4556454C53
:102B300041555820524C5920494E56414C49442049
:102B400020494E56414C49442054494D455220207D
:102B5000202056414C49442054494D4552202020C4
:102B60002020444953504C41592054494D45202080
:102B7000204348415241435445522054494D452039
:102B8000202020202020202020202020313D454EC4
:102B900020202020202020202020203130204D53B4
:102BA00020202020202020202020313030204D5394
:102BB000202020202020202020202020205345439A
:102BC0002020202020202020202020524154494F26
:102BD0000F3132333435360A6314FF320505050AE6
:102BE00000000000000000000000000000000000E5
:102BF0000000000020202020202020202020202055
:0B2C0000202020202020202020200089
:106D4B00755C64E4900000F030470B304624126B06
:106D5B000A1237E880F530480B304616126B491291
:106D6B0037E880F530490B304608123D501237E8B2
:036D7B0080F5227E
:1037E800E55C7012900000E0D394004009C247C223
:1037F80048C249C24622900000E012530238FF0036
:10380800390201390502390803390B04390D053924
:103818000F0639110739140839170A391A0B391DD7
:103828000F392010392314392615392919392C1A3A
:10383800392F1B39321E39351F393823393B243982
:103848003E2839412939442D39472E394A2F394DD7
:1038580030395032395333395534395835395B6436
:10386800395E6539616639646739676E39696F39F8
:103878006B7039AD71396D78396F7939717A39ADC5
:103888007B397382397583397784397985397C8CAA
:10389800397F8D39818E39838F3986963989973961
:1038A8008B98398D993990A03993A13996A2399876
:1038B800A3399BAA399DAB39A0AC39A2AD39A5B4BF
:1038C80039A8B539ABB639ADB739AFBE39B2BF399A
:1038D800B5C039B8C139ADC239BEF039C1F139C442
:1038E800F239C7FA39CAFB39CDFC39D0FD39D3FED4
:1038F80039D6FF000039D9027124026FC1026A4B20
:10390800026EC88004800280000267D0023EBE02B8
:103918006D7E0245940265090246E202655B024833
:1039280030026A8C026293024D6802669D02497EEB
:1039380002681A024ACC026864024C1A026E4102FA
:103948006BFD026A091268AE0263A58000025EF38D
:103958000269830265AD02693F026D150263FF804B
:10396800468032804B8040802280458007802680B8
:103978003F026784025328801C80350265FE025985
:10398800E88008802B026ACB0254A8025E158020CA
:103998000253E88012025B5C80160242EC025A6510
:1039A800025FCD800B800C025C4B02664E02569D76
:1039B800026B880264B3026EEF0260360271330252
:1039C80064590271DB0271DC0271DD025E840271EE
:0739D800DEE4900000F02284
:0F712400E4900002F0755C64900000E004F0223B
:106FC10012368A1236997BFF7A27793C126DB57F8A
:0F6FD10011123670C24DC24A900000E004F02247
:106A4B00304A3D900001E0FFC24ABF2A0790000088
:106A5B00E004F022EF642370277F2312364190006D
:106A6B0002E004F0E0C394034010C247C248C2499D
:106A7B00C246E4900000F0026C6F9000007402F0CC
:016A8B0022E8
:106EC8007BFF7A27793C126DB51236997F111236FD
:106ED8007012716BE490003CF07F2A123641C24D6B
:076EE800900000E004F0221D
:1067D000304A46900001E0F57AC24AE57A642A60C0
:1067E00038AF7A1271425022AF7A12364190003C93
:1067F000E02403F582E43400F583E57AF090003C70
:10680000E004F0900000E004F0227BFF7A27796C2E
:09681000126DB590000074FAF05D
:01681900225C
:103EBE00204A03024028900001E0FFC24ABF2A07B1
:103ECE009000007403F022EF642360030240191285
:103EDE003641900004E064397077A3E06439707164
:103EEE00A3E06439706BD24E900003E0FFB431084A
:103EFE00E4900036F0023F88EFB43208E4900037C9
:103F0E00F0023F9BEFB43302803E900003E0FFB41B
:103F1E003408E4900038F0023FC9EFB43508E4905D
:103F2E000039F0023FDFEFB43608E490003AF002B9
:103F3E003FF5EFB437028010900003E0B4380280F2
:103F4E0007900003E0B4390B7BFF7A27797C02409F
:103F5E001FC24E900003E0FFB43016A3E0B4301140
:103F6E00A3E0B4300CA3E0B43007900000740AF064
:103F7E0022EFB4310C1262365007900000740FF02D
:103F8E0022900003E0B4320C1261D650079000006C
:103F9E007414F022900003E0B43311A3E0B4300C9B
:103FAE00126F6050079000007419F022900003E029
:103FBE00B4340FA3E0B4300A127074900000741E73
:103FCE00F022900003E0B4350FA3E0B4300A127073
:103FDE00899000007423F022900003E0B4360FA302
:103FEE00E0B4300A12709E9000007428F022900007
:103FFE0003E0B43716A3E0B43011A3E0B4300CA341
:10400E00E0B43007900000742DF0227BFF7A277900
:0A401E006C126DB590000074FAF00A
:014028002275
:106D7E0090003B740BF090003C7407F0E4900049D7
:106D8E00F090004AF090004BF07BFF7A26793C128F
:106D9E006DB5126DE07F1E1236709000007432F0E9
:016DAE0022C2
:10459400125CC0D39000A7E0940A9000A6E09400B7
:1045A400400A126DAF90000074FAF0229000A6E069
:1045B400FEA3E0FF9029E975F0091252F6EE75F0BA
:1045C40009A42583F583E493900040F09029EA75CB
:1045D400F009EF1252F6EE75F009A42583F583E491
:1045E40093900041F09000A6A3E09029EB75F009A8
:1045F4001252F6EE75F009A42583F583E493900036
:1046040042F09029EC75F009EF1252F6EE75F009BC
:10461400A42583F583E493900043F09000A6A3E0DF
:104624009029ED75F0091252F6EE75F009A4258370
:10463400F583E493FD900044F09029EE75F009EFC2
:104644001252F6EE75F009A42583F583E4939000E5
:1046540045F09000A6A3E09029EF75F0091252F6F8
:10466400EE75F009A42583F583E493900046F09059
:1046740029F075F009EF1252F6EE75F009A42583BE
:10468400F583E493900047F09000A6A3E09029F10D
:1046940075F0091252F6EE75F009A42583F583E44A
:1046A40093900048F0ED6015900044E075F010A47C
:1046B4002470F9742A35F0FA7BFF126DB590004529
:1046C400E0FF601175F010A42470F9742A35F0FA33
:0E46D4007BFF126DE6900040E0900000F022A7
:1065090090003B7410F090003C7407F0E49000494F
:10651900F090004AF0900036E090004BF07BFF7A53
:1065290026794C126DB5126DE07F0D123670900010
:1065390004E0FF123641900005E0FF123641900059
:1065490006E0FF1236417F1E123670900000743249
:02655900F0222E
:1046E200125CC0D39000A7E094009000A6E0940072
:1046F200400A126DAF90000074FAF0229000A6E01A
:10470200FEA3E0FF90231075F0091252F6EE75F049
:1047120009A42583F583E493900040F0902311755A
:10472200F009EF1252F6EE75F009A42583F583E441
:1047320093900041F09000A6A3E090231275F00937
:104742001252F6EE75F009A42583F583E4939000E6
:1047520042F090231375F009EF1252F6EE75F0094C
:10476200A42583F583E493900043F09000A6A3E090
:1047720090231475F0091252F6EE75F009A4258300
:10478200F583E493FD900044F090231575F009EF52
:104792001252F6EE75F009A42583F583E493900096
:1047A20045F09000A6A3E090231675F0091252F688
:1047B200EE75F009A42583F583E493900046F0900A
:1047C200231775F009EF1252F6EE75F009A425834E
:1047D200F583E493900047F09000A6A3E09023189D
:1047E20075F0091252F6EE75F009A42583F583E4FB
:1047F20093900048F0ED6015900044E075F010A42D
:10480200242CF9742535F0FA7BFF126DB590004522
:10481200E0FF601175F010A4242CF9742535F0FA2C
:0E4822007BFF126DE6900040E0900000F02257
:10655B0090003B7415F090003C7407F0E4900049F8
:10656B00F090004AF0900037E090004BF07BFF7A00
:10657B0026795C126DB5126DE07F0C1236709000AF
:10658B0004E0FF123641900005E0FF123641900007
:10659B0006E0FF1236417F1E1236709000007432F7
:0265AB00F022DC
:10483000125CC0D39000A7E094009000A6E0940022
:10484000400A126DAF90000074FAF0229000A6E0CA
:10485000FEA3E0FF90236A75F0091252F6EE75F0A0
:1048600009A42583F583E493900040F090236B75B1
:10487000F009EF1252F6EE75F009A42583F583E4F2
:1048800093900041F09000A6A3E090236C75F0098E
:104890001252F6EE75F009A42583F583E493900097
:1048A00042F090236D75F009EF1252F6EE75F009A3
:1048B000A42583F583E493900043F09000A6A3E041
:1048C00090236E75F0091252F6EE75F009A4258357
:1048D000F583E493FD900044F090236F75F009EFA9
:1048E0001252F6EE75F009A42583F583E493900047
:1048F00045F09000A6A3E090237075F0091252F6DF
:10490000EE75F009A42583F583E493900046F090BA
:10491000237175F009EF1252F6EE75F009A42583A4
:10492000F583E493900047F09000A6A3E0902372F3
:1049300075F0091252F6EE75F009A42583F583E4AB
:1049400093900048F0ED6015900044E075F010A4DD
:10495000244CF9742535F0FA7BFF126DB5900045B3
:10496000E0FF601175F010A4244CF9742535F0FABD
:0E4970007BFF126DE6900040E0900000F02208
:106A8C007BFF7A26796C126DB57BFF7A27794C12D5
:106A9C006DE67F0E123670900005E0FF12364190C5
:106AAC000006E0FF1236417F1A12367090003B74DC
:0F6ABC001AF090003C7404F09000007432F02245
:10629300304F079000007403F022126DE07F1E124E
:1062A300367012616F9000A8E0FEA3E0FFD3940064
:1062B300EE9400402DEF94FBEE9400502590003BAC
:1062C300741BF090003C7407F0E4900049F09000D8
:1062D3004AF0900035E01490004BF09000007432C7
:0C62E300F022126DAF90000074FAF0225F
:104D6800D39000A7E094009000A6E09400400A12B7
:104D78006DAF90000074FAF0229000A6E0FEA3E068
:104D8800FF9023C475F0091252F6EE75F009A425B8
:104D980083F583E493900040F09023C575F009EF04
:104DA8001252F6EE75F009A42583F583E49390007A
:104DB80041F09000A6A3E09023C675F0091252F6C0
:104DC800EE75F009A42583F583E493900042F090F2
:104DD80023C775F009EF1252F6EE75F009A4258382
:104DE800F583E493900043F09000A6A3E09023C8D5
:104DF80075F0091252F6EE75F009A42583F583E4DF
:104E080093FD900044F09023C975F009EF1252F613
:104E1800EE75F009A42583F583E493900045F0909E
:104E280000A6A3E09023CA75F0091252F6EE75F0B9
:104E380009A42583F583E493900046F09023CB756D
:104E4800F009EF1252F6EE75F009A42583F583E414
:104E580093900047F09000A6A3E09023CC75F0094A
:104E68001252F6EE75F009A42583F583E4939000B9
:104E780048F0ED6015900044E075F010A4246CF93A
:104E8800742535F0FA7BFF126DB5900045E0FF60A0
:104E98001175F010A4246CF9742535F0FA7BFF1213
:0B4EA8006DE6900040E0900000F0225A
:10669D0090003B741FF090003C7407F0900049741B
:1066AD0064F090004A7417F0900038E090004BF0C1
:1066BD007BFF7A26797C126DB5126DE07F0F123655
:1066CD0070900005E0FF123641900006E0FF123693
:0D66DD00417F1E1236709000007432F022D2
:10497E00125CC0D39000A7E094039000A6E09400D0
:10498E00400A126DAF90000074FAF0229000A6E07B
:10499E00FEA3E0FF90241E75F0091252F6EE75F09C
:1049AE0009A42583F583E493900040F090241F75AD
:1049BE00F009EF1252F6EE75F009A42583F583E4A3
:1049CE0093900041F09000A6A3E090242075F0098A
:1049DE001252F6EE75F009A42583F583E493900048
:1049EE0042F090242175F009EF1252F6EE75F0099F
:1049FE00A42583F583E493900043F09000A6A3E0F2
:104A0E0090242275F0091252F6EE75F009A4258352
:104A1E00F583E493FD900044F090242375F009EFA4
:104A2E001252F6EE75F009A42583F583E4939000F7
:104A3E0045F09000A6A3E090242475F0091252F6DA
:104A4E00EE75F009A42583F583E493900046F0906B
:104A5E00242575F009EF1252F6EE75F009A42583A0
:104A6E00F583E493900047F09000A6A3E0902426EF
:104A7E0075F0091252F6EE75F009A42583F583E45C
:104A8E0093900048F0ED6015900044E075F010A48E
:104A9E00248CF9742535F0FA7BFF126DB590004524
:104AAE00E0FF601175F010A4248CF9742535F0FA2E
:0E4ABE007BFF126DE6900040E0900000F022B9
:10681A0090003B7424F090003C7407F0E490004927
:10682A00F090004AF0900039E090004BF07BFF7A3C
:10683A0026798C126DB5126DE07F0F1236709000BA
:10684A0005E0FF123641900006E0FF1236417F1E36
:0A685A001236709000007432F02234
:104ACC00125CC0D39000A7E094009000A6E0940084
:104ADC00400A126DAF90000074FAF0229000A6E02C
:104AEC00FEA3E0FF90247875F0091252F6EE75F0F3
:104AFC0009A42583F583E493900040F09024797504
:104B0C00F009EF1252F6EE75F009A42583F583E453
:104B1C0093900041F09000A6A3E090247A75F009E0
:104B2C001252F6EE75F009A42583F583E4939000F8
:104B3C0042F090247B75F009EF1252F6EE75F009F5
:104B4C00A42583F583E493900043F09000A6A3E0A2
:104B5C0090247C75F0091252F6EE75F009A42583A9
:104B6C00F583E493FD900044F090247D75F009EFFB
:104B7C001252F6EE75F009A42583F583E4939000A8
:104B8C0045F09000A6A3E090247E75F0091252F631
:104B9C00EE75F009A42583F583E493900046F0901C
:104BAC00247F75F009EF1252F6EE75F009A42583F7
:104BBC00F583E493900047F09000A6A3E090248046
:104BCC0075F0091252F6EE75F009A42583F583E40D
:104BDC0093900048F0ED6015900044E075F010A43F
:104BEC0024ACF9742535F0FA7BFF126DB5900045B5
:104BFC00E0FF601175F010A424ACF9742535F0FABF
:0E4C0C007BFF126DE6900040E0900000F02269
:1068640090003B7429F090003C7407F0E4900049D8
:10687400F090004AF090003AE090004BF07BFF7AF1
:1068840026799C126DB5126DE07F0D123670900062
:1068940005E0FF123641900006E0FF1236417F1EEC
:0A68A4001236709000007432F022EA
:104C1A00125CC0D39000A7E094009000A6E0940034
:104C2A00400A126DAF90000074FAF0229000A6E0DC
:104C3A00FEA3E0FF9024D275F0091252F6EE75F049
:104C4A0009A42583F583E493900040F09024D3755A
:104C5A00F009EF1252F6EE75F009A42583F583E404
:104C6A0093900041F09000A6A3E09024D475F00937
:104C7A001252F6EE75F009A42583F583E4939000A9
:104C8A0042F09024D575F009EF1252F6EE75F0094C
:104C9A00A42583F583E493900043F09000A6A3E053
:104CAA009024D675F0091252F6EE75F009A4258300
:104CBA00F583E493FD900044F09024D775F009EF52
:104CCA001252F6EE75F009A42583F583E493900059
:104CDA0045F09000A6A3E09024D875F0091252F688
:104CEA00EE75F009A42583F583E493900046F090CD
:104CFA0024D975F009EF1252F6EE75F009A425834E
:104D0A00F583E493900047F09000A6A3E09024DA9C
:104D1A0075F0091252F6EE75F009A42583F583E4BD
:104D2A0093900048F0ED6015900044E075F010A4EF
:104D3A00241CF9742635F0FA7BFF126DB5900045F4
:104D4A00E0FF601175F010A4241CF9742635F0FAFE
:0E4D5A007BFF126DE6900040E0900000F0221A
:106E41003049079000007401F02290003B742EF04D
:106E510090003C7407F07BFF7A2679AC126DB51275
:0E6E61006DE07F1E1236709000007432F02239
:106BFD00304F07900000742FF02290000AE06438A7
:106C0D006005A3E0B4390A126DAF90000074FAF07C
:106C1D00227BFF7A27795C126DB590000AE0540F44
:096C2D00F5569000007430F022CD
:106A090090000AE064386005A3E0B4390A126DAF5A
:106A190090000074FAF0227BFF7A2679BC126DB5DA
:106A290090000AE0540FF556D202D20A752EFF12D1
:106A39003BB67BFF7A27798C126DB590000074FE06
:026A4900F02239
:1068AE0090000AE0540FF556304702D200123BC852
:1068BE00304719202B04E54470F9123BBF7BFF7A59
:1068CE0027798C126DB590000074FEF030481920B7
:1068DE002904E54470F9123BBF7BFF7A27798C12AD
:0968EE006DB590000074FEF0226B
:1063A500304A56900001E0FF900034F0C24A1236A0
:1063B50041900034E0FF1271425021900034E0FF1B
:1063C50090003CE02403F582E43400F583EFF0907F
:1063D500003CE004F0900000E004F022900034E07E
:1063E500B42A079000007403F0227BFF7A27796CAA
:0A63F500126DB590000074FAF0225A
:105EF300304A6A900001E0FF900034F0C24A123643
:105F030041900034E0FFB42A0B90003BE090000086
:105F1300F0D24F22EFB4230B90003BE0900000F04F
:105F2300C24F22900034E0FF12714250219000349E
:105F3300E0FF90003CE02403F582E43400F583EFB6
:105F4300F090003CE004F0900000E004F0227BFFBE
:0E5F53007A27796C126DB590000074FAF02276
:10698300304A3F900001E0FF900034F0123641C2DC
:106993004A900034E0FFB42A0B90003BE0900000E3
:1069A300F0D24F22EFB4230B90003BE0900000F0B5
:1069B300C24F227BFF7A27796C126DB59000007469
:0369C300FAF022C5
:0A65AD00900043E0FF7003304F3808
:1065B700123670126F3D1258998F7A900041E0524F
:1065C7007AE57A60047F3180027F30123641304F9E
:1065D70017C24FE57A2430900023F09000337401FE
:0865E700F090000074F0F022B6
:0F65EF00900046E0FF123670900000E004F022AA
:10693F00304A40900001E0FF900034F0C24A123616
:10694F0041900034E0FFB42A079000007403F02256
:10695F00127142500F900034E090000DF090000043
:10696F00E004F0227BFF7A27796C126DB59000005E
:04697F0074FAF02294
:106D1500304A32900001E0FF900034F0C24ABF2AA9
:106D2500079000007403F022900034E0B42307902C
:106D35000000E004F0227BFF7A27796C126DB59094
:066D4500000074FAF022C8
:1063FF00126F3D9000AAEEF0A3EFF01258998F7A2A
:10640F0090003D7401F090000DE0B4310890004110
:10641F00E0427A800E90000DE0B4301E900041E013
:10642F00F4527A9000AAE0FEA3E0FFAD7A12585C16
:10643F001270B390000074FEF0227BFF7A27796C04
:09644F00126DB590000074FAF022
:016458002221
:105C4B00900043E0FF7003304F56123670126F3DD9
:105C5B009000AAEEF0A3EFF0E4F57A900041E0FF9C
:105C6B00E57AC39F50279000AAE475F0011252E029
:105C7B00AFF0FE1258998F7B7423257AF582E434AA
:105C8B0000F583E57BF0123641057A80CE304F105C
:105C9B00C24FE57A04900033F090000074F0F022CC
:105CAB0090003C740AF0900046E0FF1236709000B2
:045CBB0000E004F011
:015CBF0022C2
:105B5C00304A75900001E0FF900034F0C24A1236D2
:105B6C0041900034E0FFB42A079000007403F02247
:105B7C00EFB42308900000E004F080391271425019
:105B8C0038900034E0FF90003CE0FE04F074032EEB
:105B9C00F582E43400F583EFF0900041E02409FF36
:105BAC00E433FE90003CE0D39FEE6480F874809860
:105BBC004016900000E004F0227BFF7A27796C12EB
:095BCC006DB590000074FAF0229E
:106B8800304A37900001E0FF900034F0C24A1236D4
:106B980041900034E0FFB42A079000007403F0220B
:106BA800EFB42307900000E004F0227BFF7A2779F6
:0B6BB8006C126DB590000074FAF02222
:1064B300126F3D9000AAEEF0A3EFF090003C740A37
:1064C300F0E4F57A900041E0FFE57AC39F5027900E
:1064D30000AAE475F0011252E0AFF0FE90003CE038
:1064E300FD04F074032DF582E43400F583E0FD121E
:1064F300585C057A80CE7BFF7A27798C126DB59034
:05650300000074FEF031
:016508002270
:105E1500304A6B900001E0FF900034F0C24A123620
:105E250041900034E0FFB42A079000007403F0228B
:105E3500127142501A900034E0FF90003CE0FE04DD
:105E4500F074032EF582E43400F583EFF080107BC7
:105E5500FF7A27796C126DB590000074FAF02290E4
:105E65000041E02409FFE433FE90003CE0D39FEEBF
:0F5E75006480F87480984006900000E004F022EA
:10532800900043E0FF7006204F030253D3123670FB
:10533800126F3D9000AAEEF0A3EFF01258991234C4
:105348002B900041E0B401109000A3E0FF12364119
:105358009000A3E0900023F0900041E0B402209078
:1053680000A2E0FF1236419000A3E0FF1236419000
:1053780000A2E0900023F09000A3E0900024F090B9
:105388000041E0640370309000A1E0FF12364190C4
:1053980000A2E0FF1236419000A3E0FF12364190D0
:1053A80000A1E0900023F09000A2E0900024F0908B
:1053B80000A3E0900025F0304F11C24F900041E06B
:1053C800900033F090000074F0F022900046E0FF67
:1053D80012367090003C740AF0900000E004F0224D
:106784001234815002803B1234598F7A900047E0D2
:10679400FFE57AC39F402B900048E0FFE57AD39F42
:1067A4005020126F3D9000AAEEF0A3EFF0AD7A12E4
:1067B400585C7BFF7A27798C126DB590000074FECB
:0B67C400F022126DAF90000074FAF09C
:0167CF0022A7
:1065FE001234815002803F1234598F7A900047E056
:10660E00FFE57AC39F400B900048E0FFE57AD39FE9
:10661E004004E57A7020126F3D9000AAEEF0A3EFD1
:10662E00F0AD7A12585C7BFF7A27798C126DB5909B
:0F663E00000074FEF022126DAF90000074FAF0AD
:01664D00222A
:1059E800900043E0FF7003304F5E123670126F3D37
:1059F8009000AAEEF0A3EFF01258998F7A1258E2AD
:105A0800E4F57A74A1257AF582E43400F583E0FFA1
:105A18007423257AF582E43400F583EFF074A12528
:105A28007AF582E43400F583E0FF123641057AE521
:105A38007AC3940440CD304F0FC24F9000337403A3
:105A4800F090000074F0F022900046E0FF123670EB
:0C5A580090003C740AF0900000E004F0A4
:015A6400221F
:106ACB007F0A124FBB8F7AE57A6012126F3D9000EE
:106ADB00AAEEF0A3EFF0E57A14FD12585CE57A7B91
:106AEB00FF600E7A27798C126DB590000074FEF062
:0E6AFB00227A27790C126DB590000074FAF023
:016B09002269
:1054A800900043E0FF7006204F0302554312367008
:1054B800126F3D9000AAEEF0A3EFF0125899123443
:1054C8002B9000AAE475F0011252E0AFF0FE1258DA
:1054D8009912340F9000A2E0FF900023F0A3F0127D
:1054E80036419000A3E0FF1236419000AAE475F01F
:1054F800011252E0AFF0FE12589912340F9000A139
:10550800E0FF900025F09000A2E0900026F09000C7
:10551800A3E0900027F01236419000A2E0FF123677
:10552800419000A3E0FF123641304F0FC24F900068
:10553800337405F090000074F0F022900046E0FF0C
:1055480012367090003C740AF0900000E004F022DB
:1053E80090000DE0540F75F00AA4FFA3E0540F2FAE
:1053F800F57A900010E0540F75F00AA4FDACF09017
:10540800000FE0540F75F064A42DFFE5F03CFE900A
:105418000011E0540F7C002FFFEC3EFEE57AC394A8
:10542800014019E57AD394145012C3EF9401EE9415
:10543800004009D3EF94FAEE9400400A126DAF9041
:10544800000074FAF022126F3D9000AAEEF0A3EF6C
:10545800F09000AAE475F0011252E0AFF0FEAD7AC8
:1054680012585C900010E0540F75F00AA4FF9000E9
:105478000FE0540F75F064A42FFF900011E0540F53
:105488002FF57A9000AAE0FEA3E0FFAD7A12585CEF
:0F5498007BFF7A27798C126DB590000074FEF0BF
:0154A70022E2
:1042EC007F0D124FBBEF701A900010E0B43010A38A
:1042FC00E0B4300BA3E0B43006A3E06430600302FA
:10430C0043E5900014E0FF64306004EFB4350E9088
:10431C000015E0540FD3940540030243E5900014BC
:10432C00E0FF64316004EFB43611900019E0B42062
:10433C0007900018E0B420030243E5900014E0FF5E
:10434C0064326004EFB43711900018E0B420079089
:10435C000017E0B420030243E5900014E0FF64333F
:10436C006004EFB43809900015E0B42002806A9024
:10437C000014E0FF64346005EF643970669000153A
:10438C00E0540F75F00AA4FFA3E0540F2FF57A90B8
:10439C000018E0540F75F00AA4FDACF0900017E083
:1043AC00540F75F064A42DFFE5F03CFE900019E06D
:1043BC00540F7C002FFFEC3EFEE57AC394014019AC
:1043CC00E57AD394145012C3EF9401EE9400400993
:1043DC00D3EF94FAEE9400400A126DAF9000007483
:1043EC00FAF022126F3D9000AAEEF0A3EFF09000CD
:1043FC003C740AF0E4F57A900041E0FFE57AC39F43
:10440C0050279000AAE475F0011252E0AFF0FE9034
:10441C00003CE0FD04F074032DF582E43400F583D8
:10442C00E0FD12585C057A80CE7BFF7A27798C12DE
:08443C006DB590000074FEF064
:014444002255
:105A6500900043E0FF7003304F5B123670126F3DBC
:105A75009000AAEEF0A3EFF0E4F57A900041E0FF84
:105A8500E57AC39F502C9000AAE475F0011252E00C
:105A9500AFF0FE1258998F7B7423257AF582E43492
:105AA50000F583E57BF07E00125899123641057AA0
:105AB50080C9304F10C24FE57A04900033F0900052
:105AC5000074F0F022900046E0FF12367090003C22
:0B5AD500740AF0D24D900000E004F0D5
:015AE00022A3
:105FCD00304A65900001E0FF900034F0C24ABF2ACC
:105FDD00079000007403F022900034E0FFB4230812
:105FED00900000E004F0803DEF547FFF12364190A9
:105FFD000034E0547FFF90003CE0FE04F074032E6B
:10600D00F582E43400F583EFF0900041E02409FFC0
:10601D00E433FE90003CE0D39FEE6480F8748098EA
:09602D004006900000E004F0229E
:10664E00304A4B900001E0FF900034F0C24ABF2A5E
:10665E00079000007403F022900034E0FFB4230B87
:10666E00900000E004F0E004F08010127142500F30
:10667E00900034E090003EF0900000E004F0227BA9
:0F668E00FF7A27796C126DB590000074FAF02234
:10569D00204A03025739900001E0FF900034F0C218
:1056AD004ABF2A079000007403F022900034E0FFF7
:1056BD00B4230A900000E004F0E004F022127142DD
:1056CD00505B90003EE0540F75F00AA4FF9000343B
:1056DD00E0540F2FF0E090298593FF900034F012E5
:1056ED003641900034E0FF90003CE0FE04F074037E
:1056FD002EF582E43400F583EFF0900041E02409AB
:10570D00FFE433FE90003CE0D39FEE6480F874809C
:10571D0098900000E0400304F02214F0227BFF7A01
:0D572D0027796C126DB590000074FAF0221F
:106EEF003047099000B5E0F55B123335304903E4C4
:106EFF00F55B30480B304505755B0A8003755B28E1
:076F0F00900000E004F022F5
:10603600E55B70641250A9900040E012530260665E
:1060460064606B6E606B78606B82606B8C60709660
:106056006075A0607AAA607FB46084BE0000608725
:10606600127047801C126E1180171271DF80121297
:1060760071E0800D1271E180081271E280031271E5
:10608600E330470E9000B4E0787FF6900000E0041D
:09609600F0229000007401F022D8
:0F713300787FE6700912333B9000007401F02260
:1064590030470D9000B5E0F55B123335E55B70FC14
:10646900304807755B05E55B70FCE4F57A30480C4C
:1064790012719B1233DA1271CA1233DA30470C12D5
:1064890071A61233DA1271CA1233DA057AE57AC3C0
:10649900940540D930470C9000B4E0787FF6787FB6
:0964A900E670FB9000007401F0A4
:0164B20022C7
:0171DB002291
:0171DC002290
:0171DD00228F
:105E840030480A2045079000007401F02230470D85
:105E94009000B5E0F55B123335E55B70FC304807E4
:105EA400755B05E55B70FC3047151271A6E4F57A65
:105EB4001233DA057AE57AC3940A40F41271CA30CF
:105EC400481512719BE4F57A1233DA057AE57AC340
:105ED400940A40F41271CA30470C9000B4E0787F01
:0E5EE400F6787FE670FB126C6FE4900000F021
:015EF200228D
:0171DE00228E
:106B0A00302B3B204A38755C64E54B547FFF90225A
:106B1A00F093900001F0304D0EE54B30E709EF900D
:106B2A00230093900001F0D24AC22B900001E0B4F6
:0F6B3A002307900002E004F022E4900002F02212
:106B490030293B204A38755C64E549547FFF90221F
:106B5900F093900001F0304D0EE54930E709EF90D0
:106B6900230093900001F0D24AC229900001E0B4B9
:0F6B79002307900002E004F022E4900002F022D3
:103D5000204B03023EBD304A03023EBD900002E00C
:103D6000F57AE4F0755C641271D8D24ABF300790DE
:103D700000017430F022BF31079000017431F0224D
:103D8000BF32079000017432F022BF330790000168
:103D90007433F022BF34079000017434F022BF3531
:103DA000079000017435F022BF3607900001743689
:103DB000F022BF37079000017437F022BF38079018
:103DC00000017438F022BF39079000017439F022E5
:103DD000BF23109000017423F0AF7A057A9000029F
:103DE000EFF022BF2A07900001742AF022BF41079A
:103DF0009000017441F022BF42079000017442F02C
:103E000022BF43079000017443F022BF6407900073
:103E1000017444F022204D03C24A22BF6107900082
:103E2000017461F022BF62079000017462F022BF4A
:103E300063079000017463F022BF6407900001746F
:103E400064F022BF65079000017465F022BF660729
:103E50009000017466F022BF67079000017467F05C
:103E600022BF68079000017468F022BF69079000C4
:103E7000017469F022BF6A07900001746AF022BFE2
:103E80006B07900001746BF022BF6C079000017407
:103E90006CF022BF6D07900001746DF022BF6E07B9
:103EA000900001746EF022BF6F07900001746FF0F4
:0D3EB00022BF70079000017470F022C24A1A
:013EBD0022E2
:0B716B007F209000037420F0A3DFFCE5
:0171760022F6
:0F714200EFC394304007EFD39439500122C3229A
:105CC00090000CE0FD6420602E90000BE0540F75F6
:105CD000F00AA4FBAAF090000AE0540F75F064A447
:105CE0002BFFE5F03AFEED540F7C002FFFEC3E90C9
:105CF00000A6F0A3EF803190000BE0FD642090003F
:105D00000A601AE0540F75F00AA4FFED540F7C00EE
:105D10002FFEEC35F09000A6F0A3CE800BE0540FE0
:105D2000FF9000A6E4F0A3EFF0E024FFF09000A6BF
:055D3000E034FFF02249
:10616F00900009E0FD6420602B900008E0540F754B
:10617F00F00AA4FBAAF0900007E0540F75F064A496
:10618F002BFFE5F03AFEED540F7C002FFFEC3E9015
:10619F0000A8802E900008E0FD6420900007601A90
:1061AF00E0540F75F00AA4FFED540F7C002FFEECA6
:1061BF0035F09000A8F0A3CEF022E0540FFF90002E
:0761CF00A8E4F0A3EFF022A9
:106F6000900005E0540F75F00AA4FFA3E0540F2F22
:106F7000900035F0D394004006E09415500122C3F0
:016F800022EE
:10623600E4FFEF75F003A4249CF582E43427F5838C
:10624600E493FE900004E0FDEE6D703BEF75F00305
:10625600A4249DF582E43427F583E493FE9000059B
:10626600E0FDEEB50521EF75F003A4249EF582E46A
:106276003427F583E493FE900006E0FDEEB50507AE
:0C628600900036EFF0D3220FBF33A7C307
:0162920022E9
:1061D600E4FF75F003EFA42435F582E5F03428F5E5
:1061E60083E493FE900004E0FDEE6D703D75F003D0
:1061F600EFA42436F582E5F03428F583E493FE9087
:106206000005E0FDEEB5052275F003EFA42437F591
:1062160082E5F03428F583E493FE900006E0FDEE77
:0F622600B50507900037EFF0D3220FBF70A4C368
:016235002246
:104FBB0074032FF582E43400F583E0FD64317069EE
:104FCB00FE74042FF582E43400F583E0FCEE75F0FB
:104FDB0003A4249CF582E43427F583E4936C70429C
:104FEB0074052FF582E43400F583E0FCEE75F003D5
:104FFB00A4249DF582E43427F583E493B50423744C
:10500B00062FF582E43400F583E0FCEE75F003A483
:10501B00249EF582E43427F583E493B50404EE046F
:10502B00FF220EBE339B7F0022ED6432706DFE7447
:10503B00042FF582E43400F583E0FD75F003EEA454
:10504B002435F582E5F03428F583E4936D704574CF
:10505B00052FF582E43400F583E0FD75F003EEA433
:10506B002436F582E5F03428F583E493B5052574F1
:10507B00062FF582E43400F583E0FD75F003EEA412
:10508B002437F582E5F03428F583E493B50505EE76
:0D509B002434FF220EBE70977F00227F009C
:0150A80022E5
:1058E200EFC394339000A150397431F0EF75F00397
:1058F200A4249CF582E43427F583E4939000A2F07B
:10590200EF75F003A4249DF582E43427F583E49334
:105912009000A3F0EF75F003A4249EF582E43427EF
:10592200803A7432F075F003EFA4249CF582E5F01E
:105932003427F583E4939000A2F075F003EFA424DA
:105942009DF582E5F03427F583E4939000A3F0758A
:10595200F003EFA4249EF582E5F03427F583E49367
:055962009000A4F022FA
:10707400900005E0540F75F00AA4FFA3E0540F2F0D
:05708400900038F0222D
:10708900900005E0540F75F00AA4FFA3E0540F2FF8
:05709900900039F02217
:10709E00900005E0540F75F00AA4FFA3E0540F2FE3
:0570AE0090003AF02201
:066DAF007BFF7A2679DC6F
:066DB5008B7B8A7C897DC6
:106DBB007F01123670E4F57EAB7BAA7CA97D857EC4
:106DCB008275830012525EFF123641057EE57EC34B
:046DDB00941040E4EC
:016DDF002291
:066DE0007BFF7A27792CED
:066DE6008B7B8A7C897D95
:106DEC007F11123670E4F57EAB7BAA7CA97D857E83
:106DFC008275830012525EFF123641057EE57EC31A
:046E0C00941040E4BA
:016E1000225F
:106F3D0090004BE0FF90004AE08FF0A4FF900049D5
:106F4D00E07C002FFFEC35F0FE900042E02FFFECCF
:036F5D003EFE22D3
:1070B300900044E075F010A42470F9742A35F0FAB6
:0570C3007BFF026DE6F9
:0371D8007F032210
:106FE000E4F57AAF7A7E00E57A902BD093FD1258C3
:0A6FF0005C057AE57AC3941040E9CD
:016FFA002274
:106C3600E4F57AE4F57BE57A75F017A42464FFE4BD
:106C460035F0FE7C00EF257BFFEC3EFEE57B902BCE
:106C5600F493FD12585C057BE57BC3941740D7057A
:086C66007AE57AC3946440CB87
:016C6E002203
:106F1600E4F57AAF7A7E0012589974AC257AF58238
:106F2600E43400F583EFF0057AE57AC3941040E384
:066F36009000ACE0F52420
:016F3C002232
:10704700304708900023E0FF127183304808900012
:0770570023E0FF1271772214
:106E1100E4F57A900033E0FFE57AC39F50217423B3
:106E2100257AF582E43400F583E0F57B304704FFF1
:0F6E3100127183304805AF7B127177057A80D4D8
:016E4000222F
:0171DF00228D
:0171E000228C
:0171E100228B
:0171E200228A
:0171E3002289
:0C7177001271BA1233DA1271D10233DA4D
:0C7183001271C21233DA1271D10233DA39
:1050A900E4F57AF57BF57C9000A7E02401FF9000F8
:1050B900A6E03400FEC3EF940AEE94005005A3E085
:1050C90004F57CD3EF9463EE9400404C9000A7E084
:1050D9002401FB9000A6E03400FA7C007D64AF0354
:1050E900FE12528B8F7AEF75F064A4FFC3EB9FFF1A
:1050F900EA95F0FE7C007D0A12528B8F7BA3E004B7
:10510900FFE57A75F064A4FEC3EF9EFFE57B75F0B9
:105119000AA4FEC3EF9EF57C9000A7E02401FF904E
:1051290000A6E03400FED3EF9409EE940040197C08
:10513900007D0A12528B8F7BA3E004FFE57B75F09B
:105149000AA4FEC3EF9EF57C7430257AF57A743093
:10515900257BF57B7430257CF57C304714AF7A12BA
:105169007183AF7B127183AF7C1271837F2A1271B5
:1051790083304814AF7A127177AF7B127177AF7CA5
:085189001271777F2A12717781
:0151910022FB
:106F810020202056455253494F4E20312E3020208B
:106F9100204D554C544947454E455241544F52207E
:106E6F009000C17423F0A3F0E4FF74AD2FF582E41A
:106E7F003400F583E0FE74C32FF582E43400F5830C
:0C6E8F00EEF00FBF06E49000C97423F081
:016E9B0022D4
:106C6F0012359E7F011236707BFF7A6F7991126D0C
:106C7F00B57BFF7A6F7981126DE67544147F1090A2
:106C8F000091E4F0A3DFFC7F10E54470FCE490007A
:086C9F00BFF012368A0236999B
:103BB600755500123BD150FB22755500123C5A50E8
:103BC600FB22755500123C1150FB22758400E55509
:103BD60075F003A4903BDE73023C76023C85023C02
:103BE600A3023C8C023CAF023CB6023CBE023C85C2
:103BF600023CCC023C8C023CDC023CE5023C7602F8
:103C06003C85023CF3023C8C023CFF758400E55582
:103C160075F003A4903C1E73023C76023C85023C80
:103C2600A3023C8C023CAF023CB6023C76023C85C9
:103C3600023CA3023C8C023CAF023CB6023CAF0203
:103C46003CB6023CBE023C85023D01023C8C023C75
:103C5600DC023CFF758400E55575F003A4903C67D3
:103C660073023C76023C85023CF3023C8C023CFF2C
:103C7600C2FA123D11123D11759B000555C3223043
:103C8600F9020555C32230F912E59A20E7FB123DE9
:103C960011D2FA123D11123D110555C322C2FA1274
:103CA6003D11759B040555C32275431E0555C32258
:103CB600E54370020555C322C2FA123D11123D3288
:103CC600F59B0555C322C2FA123D11123D41440728
:103CD600F59B0555C322123D23F5440555C32275B0
:103CE600840F30DE04E54470020555C322C2FA1281
:103CF6003D11759B080555C322D322C2FA123D1108
:093D0600123D414405F59B0555F1
:103D0F00C3220000000000000000000000000000BF
:103D1F0000000022903D2AE55693225A5A5A5A5AC9
:103D2F00FAFAFA903D39E556932200B45AE12D87FD
:103D3F007ADB903D48E5569322000000000000809A
:013D4F0080F3
:1018B00043544353532036332E3020202020202001
:1018C00043544353532036372E30202020202020ED
:1018D00043544353532036392E34202020202020D7
:1018E00043544353532037312E39202020202020C9
:1018F00043544353532037342E34202020202020BB
:1019000043544353532037372E30202020202020AB
:1019100043544353532037392E3720202020202092
:1019200043544353532038322E352020202020208A
:1019300043544353532038352E3420202020202078
:1019400043544353532038382E3520202020202064
:1019500043544353532039312E352020202020205A
:1019600043544353532039342E3820202020202044
:1019700043544353532039372E3420202020202035
:101980004354435353203130302E30202020202028
:101990004354435353203130332E35202020202010
:1019A0004354435353203130372E322020202020FF
:1019B0004354435353203131302E392020202020EE
:1019C0004354435353203131342E382020202020DB
:1019D0004354435353203131382E382020202020C7
:1019E0004354435353203132332E302020202020C3
:1019F0004354435353203132372E332020202020AC
:101A00004354435353203133312E3820202020209B
:101A10004354435353203133362E35202020202089
:101A20004354435353203134312E3320202020207F
:101A30004354435353203134362E3220202020206B
:101A40004354435353203135312E3420202020205D
:101A50004354435353203135362E37202020202045
:101A60004354435353203135392E38202020202031
:101A70004354435353203136322E3220202020202D
:101A80004354435353203136352E35202020202017
:101A90004354435353203136372E39202020202001
:101AA0004354435353203137312E332020202020FC
:101AB0004354435353203137332E382020202020E5
:101AC0004354435353203137372E332020202020D6
:101AD0004354435353203137392E392020202020BE
:101AE0004354435353203138332E352020202020B7
:101AF0004354435353203138362E322020202020A7
:101B00004354435353203138392E3920202020208C
:101B10004354435353203139322E38202020202083
:101B20004354435353203139362E36202020202071
:101B30004354435353203139392E3520202020205F
:101B40004354435353203230332E3520202020205D
:101B50004354435353203230362E3520202020204A
:101B60004354435353203231302E3720202020203D
:101B70004354435353203231382E3120202020202B
:101B80004354435353203232352E37202020202017
:101B90004354435353203232392E31202020202009
:101BA0004354435353203233332E362020202020F9
:101BB0004354435353203234312E382020202020E8
:101BC0004354435353203235302E332020202020DD
:101BD0004354435353203235342E312020202020CB
:101BE00020202020202020202020202020202020F5
:101BF0004443532030303620494E56203032312075
:101C00004443532030303720494E5620323134205F
:101C10004443532030313520494E56203134312051
:101C20004443532030313720494E56203035302040
:101C30004443532030323120494E56203030362034
:101C40004443532030323320494E5620303437201D
:101C50004443532030323520494E5620323434200C
:101C60004443532030323620494E562034363420F7
:101C70004443532030333120494E562036323720EA
:101C80004443532030333220494E562030353120E2
:101C90004443532030333620494E562031373220CA
:101CA0004443532030343320494E562034343520B9
:101CB0004443532030343720494E562030323320AD
:101CC0004443532030353020494E562030313720A0
:101CD0004443532030353120494E56203033322092
:101CE0004443532030353320494E5620343532207A
:101CF0004443532030353420494E5620343133206C
:101D00004443532030363520494E56203237312057
:101D10004443532030373120494E5620333036204B
:101D20004443532030373220494E56203234352038
:101D30004443532030373320494E56203530362027
:101D40004443532030373420494E56203137342015
:101D50004443532031313420494E5620373132200C
:101D60004443532031313520494E562031353220FD
:101D70004443532031313620494E562037353420E4
:101D80004443532031323220494E562032323520DE
:101D90004443532031323520494E562033363520C6
:101DA0004443532031333120494E562033363420BA
:101DB0004443532031333220494E562035343620A7
:101DC0004443532031333420494E5620323233209D
:101DD0004443532031343120494E56203031352090
:101DE0004443532031343320494E5620343132207D
:101DF0004443532031343520494E56203237342065
:101E00004443532031353220494E5620313135205C
:101E10004443532031353520494E56203733312045
:101E20004443532031353620494E56203236352032
:101E30004443532031363220494E5620353033202A
:101E40004443532031363520494E56203235312017
:101E50004443532031373220494E56203033362008
:101E60004443532031373420494E562030373420F4
:101E70004443532032303520494E562032363320E9
:101E80004443532032313220494E562033353620D8
:101E90004443532032313420494E562030303720CD
:101EA0004443532032323320494E562031333420BC
:101EB0004443532032323520494E562031323220AD
:101EC0004443532032323620494E5620343131209B
:101ED0004443532032343320494E56203335312089
:101EE0004443532032343420494E5620303235207A
:101EF0004443532032343520494E56203037322067
:101F00004443532032343620494E56203532332054
:101F10004443532032353120494E56203136352046
:101F20004443532032353220494E56203436322035
:101F30004443532032353520494E56203434362020
:101F40004443532032363120494E56203733322015
:101F50004443532032363320494E56203230352008
:101F60004443532032363520494E562031353620F1
:101F70004443532032363620494E562034353420DF
:101F80004443532032373120494E562030363520D5
:101F90004443532032373420494E562031343520C3
:101FA0004443532033303620494E562030373120B9
:101FB0004443532033313120494E562036363420A5
:101FC0004443532033313520494E56203432332098
:101FD0004443532033323520494E56203532362083
:101FE0004443532033333120494E56203436352074
:101FF0004443532033333220494E56203435352064
:102000004443532033343320494E56203533322055
:102010004443532033343620494E56203631322043
:102020004443532033353120494E56203234332037
:102030004443532033353620494E56203231322026
:102040004443532033363420494E56203133312017
:102050004443532033363520494E56203132352003
:102060004443532033373120494E562037333420F0
:102070004443532034313120494E562032323620E9
:102080004443532034313220494E562031343320DA
:102090004443532034313320494E562030353420C8
:1020A0004443532034323320494E562033313520B7
:1020B0004443532034333120494E562037323320A5
:1020C0004443532034333220494E56203531362094
:1020D0004443532034343520494E56203034332085
:1020E0004443532034343620494E5620323535206F
:1020F0004443532034353220494E56203035332066
:102100004443532034353420494E5620323636204D
:102110004443532034353520494E56203333322042
:102120004443532034363220494E56203235322033
:102130004443532034363420494E56203032362022
:102140004443532034363520494E56203333312012
:102150004443532034363620494E562036363220FA
:102160004443532035303320494E562031363220F7
:102170004443532035303620494E562030373320E3
:102180004443532035313620494E562034333220D3
:102190004443532035323320494E562032343620C2
:1021A0004443532035323620494E562033323520B1
:1021B0004443532035333220494E562033343320A4
:1021C0004443532035343620494E56203133322093
:1021D0004443532035363520494E5620373033207E
:1021E0004443532036303620494E56203633312072
:1021F0004443532036313220494E56203334362062
:102200004443532036323420494E56203633322050
:102210004443532036323720494E56203033312044
:102220004443532036333120494E56203630362031
:102230004443532036333220494E56203632342020
:102240004443532036353420494E5620373433200A
:102250004443532036363220494E562034363620F9
:102260004443532036363420494E562033313120F2
:102270004443532037303320494E562035363520DD
:102280004443532037313220494E562031313420D7
:102290004443532037323320494E562034333120C3
:1022A0004443532037333120494E562031353520B1
:1022B0004443532037333220494E562032363120A2
:1022C0004443532037333420494E5620333731208E
:1022D0004443532037343320494E5620363534207A
:1022E0004443532037353420494E5620313136206F
:1051920075840F1200A4126E6F126C6FE49003F804
:1051A200F0A3F09003F6F0A3F01270F01269C612A9
:1051B200303D1230D7126BC31271B1E54270031247
:1051C200368A30361A123111EF75F010A424B0F974
:1051D200741835F0FA7BFF126DB5C23675421E3077
:1051E2003318E55F75F010A424F0F9741B35F0FA5A
:1051F2007BFF126DB5C23375421E3056081244450C
:10520200C25675421E305305125AE1C25330522F14
:10521200C2527F0C1236B7126FE0126C36126F1642
:10522200126E6FE49000B9F0C247C248C249F579E4
:105232001233DA0579E579C3941E40F4126C6F20BB
:1052420046030251AE126D4B126F16126E6FE4904E
:0C52520000B9F0C247C248C2490251AE88
:104EB30009920A9E0BC70D100E7D101211D213C555
:104EC30015ED185208D0094E09D40A600AF40B9163
:104ED3000C360CE50D9D0E600F2D100610EB11DD49
:104EE30012DC13EA15071633177118C01D2107B119
:104EF30007E808200859196E1A211ADA1B971C5A59
:104F03000894090E09900A190AA90B410BE30C8CAA
:104F13000D3F0DFD0EC50F9810771162125B1362E2
:104F23001477159B16D018161DEF1EC21F9B2079F0
:104F3300215F224A233B24342533263912330FCDF4
:104F430014331566169A17CD19000E9A13661100BD
:104F530011661033150016331766189A19CD0DCD47
:104F63000F00129A11CD1300149A15CD17001833A0
:104F730019660E330F66109A191823A01296203D56
:104F8300129623A0129627631488203D148823A029
:104F93001488276316B8203D16B823A016B82763D4
:104FA3001918203D1918276312962B8C14882B8C03
:084FB30016B82B8C19182B8C89
:0B719B0075081575095ED22DD2032285
:0B71A60075081575095ED22DD20B2272
:0771CA00C22DC203C20B221B
:0871BA0012418BD22ED20422F7
:0871C20012418BD22ED20C22E7
:09418B00E4F512F513F514F51525
:10419400EF125302428F23427E2A41CC3041DE315A
:1041A40041F0324202334214344226354238364218
:1041B4004A37425C38426D3942A04142B14242C260
:1041C4004342D344000042EB904F7BE493F50D74DB
:1041D4000193F50E904F7D0242E2904F7FE493F5F8
:1041E4000D740193F50E904F810242E2904F83E4E7
:1041F40093F50D740193F50E904F850242E2904FB2
:1042040087E493F50D740193F50E904F890242E211
:10421400904F8BE493F50D740193F50E904F8D023E
:1042240042E2904F8FE493F50D740193F50E904F95
:10423400910242E2904F93E493F50D740193F50ECD
:10424400904F950242E2904F97E493F50D740193D9
:10425400F50E904F990242E2904F9BE493F50D7452
:104264000193F50E904F9D8075904F9FE493F50D4B
:10427400740193F50E904FA18064904FA3E493F5DD
:104284000D740193F50E904FA58053904FA7E493BE
:10429400F50D740193F50E904FA98042904FABE455
:1042A40093F50D740193F50E904FAD8031904FAF9F
:1042B400E493F50D740193F50E904FB18020904F67
:1042C400B3E493F50D740193F50E904FB5800F9000
:1042D4004FB7E493F50D740193F50E904FB9E49341
:0842E400F50F740193F510229F
:0771D100C22EC20CC2042211
:100DB700C0D0C000C001C083C082C0E0C0F0A29212
:100DC700305A01B37864E233F208E233F208E233CF
:100DD700F208E233F208E233F208E233F208E233D0
:100DE700F208E233F208E233F208E233F208E233C0
:100DF700F208E233F208E233F208E233F208E233B0
:100E0700F208E233F208E233F208E233F208E2339F
:100E1700F208E233F208E233F208E233F208E2338F
:100E2700F208E233F208E233F208E233F208E2337F
:100E3700F208E233F208E233F208E233F208E2336F
:100E4700F208E233F208E233F208E233F208E2335F
:100E5700F208E233F208E233F208E233F208E2334F
:100E6700F208E233F2901260788BE218936028E27E
:100E770018937023E21893601EE218937019E21812
:100E8700936014E21893600FE21893700AE21893C4
:100E97007005E21893600302104C756000E2189326
:100EA7001392545003756038752300E21893139218
:100EB7001C500363601CE2189313921B500363607A
:100EC7000EE2189313921A5003636046E2189313C5
:100ED70092195003636023E21893139218852361D4
:100EE7005003636051752300E2189313921C50035B
:100EF700636068E2189313921B5003636075E218EE
:100F07009313921A500363607AE21893139219505D
:100F17000363603DE21893139218852362500363BD
:100F2700601F752300E2189313921F500363604FED
:100F3700E2189313921E5003636026E218931392EC
:100F47001D5003636052E2189313921C50036360B1
:100F570029E2189313921B5003636015E218931349
:100F6700921A500363600BE21893139219500363AC
:100F77006045E218931392188523635003636062F8
:100F8700E2189313921C5003636031E21893139293
:100F97001B5003636019E2189313921A500363609E
:100FA7000DE218931392195003636007E218931325
:100FB70092188523645003636043752300E21893F6
:100FC70013921EE2189313921DE2189313921CE2D8
:100FD700189313921BE2189313921AE21893139221
:100FE70019E21893139218852365C257E565656062
:100FF7006035D25723F89017B193F99017B0E8935B
:101007006025B40104B254801EB40205E862618011
:0D10170016B40305E86262800EB40405E81B
:1010240062638006B40521E86264A254925590007C
:101034008CE561F090008DE562F090008EE563F040
:1010440090008FE564F0D25612105ED0F0D0E0D05C
:1010540082D083D001D000D0D032C0D0C000C0E054
:101064007881E6603D303133788016E6702D76085D
:101074007881167886E6A2E7304301B39241D23EE6
:10108400A2E77882E633F67883E633F67884E633AB
:10109400F67885E633F67886E633F6D0E0D000D0ED
:1010A400D0227628D0E0D000D0D022C0D0C000C05A
:1010B40001C083C082C0E0C0F0C259A2922059018D
:1010C400B3784CE213F208E213F208E213F208E2F6
:1010D40013F208E213F208E213F208E213F208E250
:1010E40013F208E213F208E213F208E213F208E240
:0D10F40013F208E213F208E213F208E2130F
:10110100F208E213F208E213F208E213F208E21322
:10111100F208E213F208E213F208E213F208E21312
:10112100F2901260784CE20893139217E20893133D
:101131009216E20893139215E20893139214E208AF
:1011410093139213E20893139212E20893139211EC
:10115100E20893139210852266E20893139217E234
:101161000893139216E20893139215E208931392CF
:1011710014E20893139213E20893139212E2089374
:10118100139211E20893139210852267E2089313D8
:101191009217E20893139216E20893139215E2084C
:1011A10093139214E20893139213E2089313921289
:0311B100E20893BE
:1011B400139211C210852268E5669015B0856722E6
:1011C400301602058393602F14F875F003A490146D
:1011D400612582F582E5F03583F583E493F9A3E490
:1011E40093901360656893C965679329B4010050AF
:1011F40006885FD233B2A312120DD0F0D0E0D082B1
:10120400D083D001D000D0D032302F26788716E694
:1012140070207608788AE6A2E1304401B3923CD289
:1012240039A2E17888E613F67889E613F6788AE637
:1012340013F622EF90146075F003A42582F582E57D
:101244008335F0F583C22F7400937888F674019384
:101254007889F6740293788AF6D22F22000000006F
:10126400000000000000000000000000000000007A
:101274000000000000000000000000010000000069
:101284000000000000000000000000010000000059
:101294000000000100000001000101010000000045
:1012A4000000000000000000000000010000000039
:1012B4000000000100000001000101010000000025
:1012C4000000000100000001000101010000000114
:1012D4000001010100010101010101010000000000
:1012E40000000000000000000000000100000000F9
:1012F40000000001000000010001010100000000E5
:1013040000000001000000010001010100000001D3
:1013140000010101000101010101010100000000BF
:1013240000000001000000010001010100000001B3
:10133400000101010001010101010101000000019E
:10134400000101010001010101010101000101018C
:101354000101010101010101010101010001010279
:101364000102020301020203020303040102020355
:10137400020303040203030303030405010202033B
:101384000203030402030304030404050203030425
:10139400030404050304040404050506010202030E
:1013A4000203030402030303030404050203030406
:1013B40003030405030404050405050602030304EA
:1013C40003040405030404050405050603040405D5
:1013D40004050506040505060506060701020203C1
:1013E40002030304020303040304040502030304C5
:1013F40003040405030404050405050602030304A9
:101404000304040503040405040505060304040594
:10141400040505060405050605060607020303047C
:101424000304040503040405040505060304040574
:101434000405050604050506050606070304040558
:101444000405050604050506050606070405050644
:10145400050606070506060706070708FDD00C73F0
:10146400700E3CF01AAF101E7F9022EC7026D6F05E
:101474002ACBB02CA3F032BEB03417D03CB6D04641
:101484001FB04E77F050F950526AB056DE9058BAF9
:10149400306ACF3072D270745CD076E8F0786BD05A
:1014A40098E5709AF8309CBB50A40F70AA7A70B279
:1014B4006730B45DB0B8FCB0C26F50C655D0CA3DF9
:1014C40090D489B0DA94F0DCD790E463B0EA0BF0FE
:1014D400F43170F8DD310AB571148FF118D1D126C9
:1014E400EB512AF6112C8B71463F5148B1F14AACAD
:1014F400B14CC4F152D9B1546D915A2EF162BD115F
:101504006687916A9AD16CF29172D5517819F18CEF
:1015140071B192D8D19A32D1AA47D1B25A91B45268
:0D152400F1C67531CC1D71D2A951DCD0B1DA
:10153100E85E11EA2B11F2EED212F392147D32160B
:10154100973226D8B232C5F234F7124AEA524C9F8A
:101551005254A5D2582B725A7552644FD268C17237
:101561006ADC326C78D2865F128C83729C4EB2A692
:101571006972AC1C72B433D2CC18F2EABB330CCE14
:1015810033141EB32803F32EE51332F85334987342
:101591005848F36472736845738617B3947313A63E
:1015A1003C93B221D3B41B53B829B3C641F3D8003D
:1015B100000000000000000000000000000000002A
:1015C1000000000000006A000000000000620D0041
:1015D10000000000000000006F0048000000000053
:1015E10000000000000000000000006C220000006C
:1015F100000000000000000000000000005B00008F
:101601000000000000000000004100001E475900DA
:101611000000260000001D00001000003500000041
:101621003D006B0043000000000000004B0005007E
:10163100000000000000380023000000000000004E
:101641000000000000004C0000000000000000004D
:101651000000000000000000000000320000040053
:10166100000000000000000000126000370A0000C6
:1016710000000000000000000000080000611346A7
:10168100000000000000254D340000572911000022
:1016910000000000640000000000000000000000E5
:1016A100003A4A00002E4F190000001F0000000000
:1016B10000006300000000000000270000001B0084
:1016C1000000000000000B5F3C006E5D4400000064
:1016D1006D00000000000000000053000036000013
:1016E100283F5E0000000000000000030000300001
:1016F1007000000069004067000000000000550014
:101701000042000021000000000000150000000060
:1017110000000000000000005C0017000000200035
:101721000068020054000E58001C00000000000078
:1017310000005A000000000000002F0000002B00F4
:101741000000002400000066003900000000510084
:1017510000000900520000004500000000000000E8
:10176100310000002A0C000000001A0000000000F7
:10177100560000334E000000000000000000000091
:101781002C1400003B07003E000000000000000098
:10179100000000001800001600502D06004900004E
:1017A10000000000000000650F00000001000000C3
:1017B1000000000000060000000600060005020609
:1017C10000060006000404060005040208060000E5
:1017D10000060006000600060004080600060006D2
:1017E10000050806000600021006000600030100BD
:1017F100000600060002020600060004400600067C
:101801000004100600060006000600060006000699
:10181100000510060006000600060006000600018D
:10182100010600060006000600030206000600008D
:101831000006000600050106000402020406000677
:1018410000060006000600060006000600048006E9
:10185100000201042006000600060006000600063C
:101861000006000600060006000600060006000647
:10187100000600040106000600060006000600033B
:101881001006000600060006000600060006000617
:101891000006000600060006000308060006000612
:0D18A1000006000304060006000600060015
:0218AE00060032
:102FE000C0E0758400C2CA85CC6F85CD6E75CC00FB
:102FF00075CD00D2CA10CF3D20343FE569B4000A38
:10300000856E70856F710569802EB4010A856E72B8
:10301000856F7305698021B4020A856E74856F75AA
:1030200005698014B4030E856E76856F77D234758A
:103030006900D0E032756900C234D0E032C0D0C03F
:10304000E0C000C001C002C003C004C005C006C08B
:103050000730346EAA71AB70AE02AF03EEC4030347
:103060005403FEEFC40303FF54FC4EFEEF5403FF72
:10307000C3E5739AFCE5729BFD50066304FF63058C
:10308000FFC3EC9EED9F5038C3E5759AFCE5749B39
:10309000FD50066304FF6305FFC3EC9EED9F5020C7
:1030A000C3E5779AFCE5769BFD50066304FF630554
:1030B000FFC3EC9EED9F500885706B85716AD23519
:1030C000C234D007D006D005D004D003D002D0013E
:1030D000D000D0E0D0D022303536903235E56B9339
:1030E000FF90316923232582F582E5833400F5833F
:0930F00012314840100F12314862
:1030F900400A0F1231484004C235800B788CE6042F
:10310900B40603D23622F622303533903235E56BD8
:1031190093FF90316923232582F582E5833400F5F5
:103129008312314840100F123148400A0F123148BA
:103139004004C2358008D236C235E4788CF622E4E0
:1031490093F9A3E493FAA3E493FBA3E493FCA3C345
:10315900E56A9AE56B995007C3EC956AEB956B2282
:10316900EA25DD89DD89D324D324CBD2CBD2C4DBB4
:10317900C4DBBE39BE39B7CAB7CAB18EB18EAB8707
:10318900AB87A59CA59CA000A0009A969A9695D875
:1031990095D891E591E58D858D8588AF88AF840CAB
:1031A900840C7F9A7F9A7B497B49771B771B730F26
:1031B900730F6F276F276B576B5767AB67AB642C20
:1031C900642C60C660C65D795D795AFE5AFE5970F5
:1031D900597057E257E25661566154E754E7537400
:1031E90053745207520750A050A04F404F404DE62C
:1031F9004DE64C934C934B414B4149F549F548B544
:1032090048B547764776463E463E45084508432A2F
:10321900432A40E440E43F533F533E3E3E3E3C9404
:103229003C943A863A86391839183805323232329E
:103239003232323232323232323232323232323265
:103249003232323232323232323232323232323255
:103259003232323232323232323232323232323245
:103269003232323232313130302F2E2D2D2D2C2C5D
:103279002B2A2929282726252524232322212020F2
:103289001F1E1E1D1C1C1B1A1A1A1A191919181887
:1032990018171717171616161615151515141414C9
:1032A90014131313131212121211111111101010F9
:1032B90010100F0F0F0F0F0E0E0E0E0E0D0D0D0C21
:1032C9000C0C0C0B0B0B0B0B0B0A0A0A0A0A09094B
:1032D9000909090908080808080807070707070767
:1032E9000606060606060605050505050504040481
:1032F9000404040403030303030303020202020296
:1033090002020101010101010101010101010101A2
:1033190000000000000000000000000000000000A4
:0C33290000000000000000000000000098
:104445007F011236707F4C1236417F541236417F00
:10445500521236417F201236412055047F308002AA
:104465007F311236417F2012364190008DE0784E23
:104475001234D2784E860743073012364108860734
:1044850043073012364175072012364190008EE001
:10449500784E1234CA784E860743073012364108E3
:1044A5008607430730123641088607430730123620
:1044B5004175072012364190008CE0784E1234D2B7
:1044C500784E860743073012364108860743073082
:1044D50012364175072012364122C007C0007F11F0
:1044E5001236707F4C12364175072012364120581E
:1044F500047F3080027F311236417F201236419091
:1045050003F2E0784E1234D2784E86074307301214
:1045150036410886074307301236417507201236A3
:10452500419003F3E0784E1234CA784E860743076C
:104535003012364108860743073012364108860790
:104545004307301236417507201236419003F4E0D7
:10455500784E1234D2784E8607430730123641081A
:1045650086074307301236417507201236419003FE
:10457500F5E0784E1234D2784E860743073012366E
:0F45850041088607430730123641D000D0072285
:1071140044313233343536373839302A2341424307
:0971B10012705E500312702F22CF
:106BC300303736E54B540F90711493FF9003F8E47C
:106BD30075F0011252E0FC74D225F0F58274003C8A
:106BE300F583EFF0C2379003F8E0B4030CA3E0B4ED
:0A6BF3002007E49003F8F0A3F0225D
:10705E009003F6E0FEA3E0FFA3E0B50607A3E0B5BC
:06706E000702C322D32239
:106E9C009003F6E475F0011252E0FE74D225F0F581
:106EAC008274003EF583E0FF9003F6E0B4030CA37C
:0B6EBC00E0B42007E49003F6F0A3F020
:016EC70022A8
:10702F009000D0E014600A14600A2402700902680C
:08703F00F7027103126FA12298
:1068F7009000C0E0FFD3940F5034EF700312369925
:10690700126E9C7895760008A6079000C0E02411C7
:10691700FF1236707896E6FF9000C0E0FE04F07430
:10692700912EF582E43400F583EFF0023641754489
:07693700329000D0E004F0F3
:01693E002236
:10710300E544700C12369975440A9000D0E004F0FF
:017113002259
:106FA100E544701B7F11123670126E9C900091EFB8
:0F6FB100F01236419000C07401F0E49000D0F06F
:016FC00022AE
:1002510043544353532036332E3020202020202076
:1002610043544353532036372E3020202020202062
:1002710043544353532036392E342020202020204C
:1002810043544353532037312E392020202020203E
:1002910043544353532037342E3420202020202030
:1002A10043544353532037372E3020202020202021
:1002B10043544353532037392E3720202020202008
:1002C10043544353532038322E3520202020202000
:1002D10043544353532038352E34202020202020EE
:1002E10043544353532038382E35202020202020DA
:1002F10043544353532039312E35202020202020D0
:1003010043544353532039342E38202020202020B9
:1003110043544353532039372E34202020202020AA
:100321004354435353203130302E3020202020209D
:100331004354435353203130332E35202020202085
:100341004354435353203130372E32202020202074
:100351004354435353203131302E39202020202063
:100361004354435353203131342E38202020202050
:100371004354435353203131382E3820202020203C
:100381004354435353203132332E30202020202038
:100391004354435353203132372E33202020202021
:1003A1004354435353203133312E38202020202011
:1003B1004354435353203133362E352020202020FF
:1003C1004354435353203134312E332020202020F5
:1003D1004354435353203134362E322020202020E1
:1003E1004354435353203135312E342020202020D3
:1003F1004354435353203135362E372020202020BB
:100401004354435353203135392E382020202020A6
:100411004354435353203136322E322020202020A2
:100421004354435353203136352E3520202020208C
:100431004354435353203136372E39202020202076
:100441004354435353203137312E33202020202071
:100451004354435353203137332E3820202020205A
:100461004354435353203137372E3320202020204B
:100471004354435353203137392E39202020202033
:100481004354435353203138332E3520202020202C
:100491004354435353203138362E3220202020201C
:1004A1004354435353203138392E39202020202002
:1004B1004354435353203139322E382020202020F9
:1004C1004354435353203139362E362020202020E7
:1004D1004354435353203139392E352020202020D5
:1004E1004354435353203230332E352020202020D3
:1004F1004354435353203230362E352020202020C0
:100501004354435353203231302E372020202020B2
:100511004354435353203231382E312020202020A0
:100521004354435353203232352E3720202020208C
:100531004354435353203232392E3120202020207E
:100541004354435353203233332E3620202020206E
:100551004354435353203234312E3820202020205D
:100561004354435353203235302E33202020202052
:100571004354435353203235342E31202020202040
:10058100202020202020202020202020202020206A
:100591004443532030303620494E562030323120EA
:1005A1004443532030303720494E562032313420D5
:1005B1004443532030313520494E562031343120C7
:1005C1004443532030313720494E562030353020B6
:1005D1004443532030323120494E562030303620AA
:1005E1004443532030323320494E56203034372093
:1005F1004443532030323520494E56203234342082
:100601004443532030323620494E5620343634206C
:100611004443532030333120494E5620363237205F
:100621004443532030333220494E56203035312057
:100631004443532030333620494E5620313732203F
:100641004443532030343320494E5620343435202E
:100651004443532030343720494E56203032332022
:100661004443532030353020494E56203031372015
:100671004443532030353120494E56203033322007
:100681004443532030353320494E562034353220EF
:100691004443532030353420494E562034313320E1
:1006A1004443532030363520494E562032373120CD
:1006B1004443532030373120494E562033303620C1
:1006C1004443532030373220494E562032343520AE
:1006D1004443532030373320494E5620353036209D
:1006E1004443532030373420494E5620313734208B
:1006F1004443532031313420494E56203731322082
:100701004443532031313520494E56203135322072
:100711004443532031313620494E56203735342059
:100721004443532031323220494E56203232352053
:100731004443532031323520494E5620333635203B
:100741004443532031333120494E5620333634202F
:100751004443532031333220494E5620353436201C
:100761004443532031333420494E56203232332012
:100771004443532031343120494E56203031352005
:100781004443532031343320494E562034313220F2
:100791004443532031343520494E562032373420DA
:1007A1004443532031353220494E562031313520D2
:1007B1004443532031353520494E562037333120BB
:1007C1004443532031353620494E562032363520A8
:1007D1004443532031363220494E562035303320A0
:1007E1004443532031363520494E5620323531208D
:1007F1004443532031373220494E5620303336207E
:100801004443532031373420494E56203037342069
:100811004443532032303520494E5620323633205E
:100821004443532032313220494E5620333536204D
:100831004443532032313420494E56203030372042
:100841004443532032323320494E56203133342031
:100851004443532032323520494E56203132322022
:100861004443532032323620494E56203431312010
:100871004443532032343320494E562033353120FE
:100881004443532032343420494E562030323520EF
:100891004443532032343520494E562030373220DC
:1008A1004443532032343620494E562035323320CA
:1008B1004443532032353120494E562031363520BC
:1008C1004443532032353220494E562034363220AB
:1008D1004443532032353520494E56203434362096
:1008E1004443532032363120494E5620373332208B
:1008F1004443532032363320494E5620323035207E
:100901004443532032363520494E56203135362066
:100911004443532032363620494E56203435342054
:100921004443532032373120494E5620303635204A
:100931004443532032373420494E56203134352038
:100941004443532033303620494E5620303731202E
:100951004443532033313120494E5620363634201A
:100961004443532033313520494E5620343233200D
:100971004443532033323520494E562035323620F8
:100981004443532033333120494E562034363520E9
:100991004443532033333220494E562034353520D9
:1009A1004443532033343320494E562035333220CB
:1009B1004443532033343620494E562036313220B9
:1009C1004443532033353120494E562032343320AD
:1009D1004443532033353620494E5620323132209C
:1009E1004443532033363420494E5620313331208D
:1009F1004443532033363520494E56203132352079
:100A01004443532033373120494E56203733342065
:100A11004443532034313120494E5620323236205E
:100A21004443532034313220494E5620313433204F
:100A31004443532034313320494E5620303534203D
:100A41004443532034323320494E5620333135202C
:100A51004443532034333120494E5620373233201A
:100A61004443532034333220494E56203531362009
:100A71004443532034343520494E562030343320FA
:100A81004443532034343620494E562032353520E4
:100A91004443532034353220494E562030353320DB
:100AA1004443532034353420494E562032363620C3
:100AB1004443532034353520494E562033333220B8
:100AC1004443532034363220494E562032353220A9
:100AD1004443532034363420494E56203032362098
:100AE1004443532034363520494E56203333312088
:100AF1004443532034363620494E56203636322070
:100B01004443532035303320494E5620313632206C
:100B11004443532035303620494E56203037332058
:100B21004443532035313620494E56203433322048
:100B31004443532035323320494E56203234362037
:100B41004443532035323620494E56203332352026
:100B51004443532035333220494E56203334332019
:100B61004443532035343620494E56203133322008
:100B71004443532035363520494E562037303320F3
:100B81004443532036303620494E562036333120E7
:100B91004443532036313220494E562033343620D7
:100BA1004443532036323420494E562036333220C6
:100BB1004443532036323720494E562030333120BA
:100BC1004443532036333120494E562036303620A7
:100BD1004443532036333220494E56203632342096
:100BE1004443532036353420494E56203734332080
:100BF1004443532036363220494E5620343636206F
:100C01004443532036363420494E56203331312067
:100C11004443532037303320494E56203536352052
:100C21004443532037313220494E5620313134204C
:100C31004443532037323320494E56203433312038
:100C41004443532037333120494E56203135352026
:100C51004443532037333220494E56203236312017
:100C61004443532037333420494E56203337312003
:100C71004443532037343320494E562036353420EF
:100C81004443532037353420494E562031313620E4
:100C910001AE01C901DA01EB01FC020E02200233AF
:100CA1000247025C02710287029902AB02C302DCB5
:100CB10002F50310032B03480365038403A403C552
:100CC10003E6040A042E04430453046A047A0491DB
:100CD10004A204BA04CC04E504F705100524053E7A
:100CE1000552056D0582059E05D10605061C063BCC
:100CF100067306AD06C744313233343536373839D9
:100D0100302A23414243202020202020202020205F
:100D1100202020202020202044435320504F4C41AC
:100D210052495459202020204C545220504F4C41BC
:100D310052495459202020204C54522041524541BF
:100D4100204249542020204C545220474F544F20D8
:100D51004649454C442020494E5445524E414C2071
:100D61004C4556454C202047454E4552415445205F
:100D71004354435353202047454E45524154452047
:100D81004443532020202047454E4552415445209D
:100D91004C545220202020494E56414C4944204970
:100DA1004E5055545320454E434F444520435443E0
:060DB100535320313030E5
:1069C600305017C250E54B547F900CF7939000CE91
:1069D600F0788B76321266EA8009788BE67004903E
:1069E60000D1F0305114C251E549547F900CF79311
:1069F6009000CDF0755832026737E5587004900361
:036A0600FAF02281
:1066EA009000D1E0B40A0050439066FAF828287363
:1066FA0002671802671B02671E02672102672402EB
:10670A00672702672A02672D026730026733026F22
:10671A00FB0270C8025D350262EF02609F026CA73D
:0D672A00025BD5025F610255FC1271512225
:106FFB009000CEE0FFB42A079000D1E004F022EF1E
:0A700B00B423069000D17405F022B2
:1070C8009000CEE0B42A079000D1E004F022E490CA
:0470D80000D1F022D1
:105D35009000CEE0B4310D7BFF7A0D7917126DB569
:105D4500B244802C9000CEE0B432107BFF7A0D79FE
:105D550027126DB5B24312573A80159000CEE0B4C4
:105D650033187BFF7A0D7937126DB5B25812573A51
:105D75007578029000D17409F0229000CEE0FFB44E
:105D8500340D90003C740AF09000D1E004F022EF4D
:105D9500B4350C90003C740AF09000D17404F022E4
:1062EF009000CEE0FF127142504B9000CEE0FF9035
:1062FF00003CE0FE04F074032EF582E43400F583D5
:10630F00EFF090003CE0D3940B402F7BFF7A0D7998
:10631F0047126DB590000DE0540F75F00AA4FFA35E
:10632F00E0540F2F9003F4F012573A757802900053
:0B633F00D17409F022E49000D1F0229C
:10609F009000CEE0FF12714250589000CEE0FF907A
:1060AF00003CE0FE04F074032EF582E43400F58327
:1060BF00EFF090003CE0D3940C403C7BFF7A0D79DD
:1060CF0057126DB590000EE0540F75F00AA4FF90B3
:1060DF00000DE0540F75F064A42FFF90000FE054F3
:1060EF000F2FF533F532F52F7578029000D1740923
:0860FF00F022E49000D1F02230
:106CA7009000CEE0FFB4310D90003C7401F09000ED
:106CB700D1E004F022EFB4320D90003C7401F09063
:106CC70000D17407F022EFB4330C90003C7401F04C
:076CD7009000D17408F022C7
:105BD5009000CEE0FF12714250599000CEE0FF9048
:105BE500003CE0FE04F074032EF582E43400F583F6
:105BF500EFF090003CE0D39403404A1262365033F4
:105C0500C22FC231C20EC20F900036E025E02491AA
:105C1500F582E4340CF583E493F516740193F517D6
:105C2500D230D20D7BFF7A0D7967126DB5E4900005
:105C3500D1F0227BFF7A0D7997126DB575780290B8
:065C450000D17409F022F9
:105F61009000CEE0FF127142504F9000CEE0FF90C2
:105F7100003CE0FE04F074032EF582E43400F58366
:105F8100EFF090003CE0D3940340401261D65029D9
:105F9100C20FC231C22DC20BC230C20D7887760842
:105FA100900037E0FF121237D20E7BFF7A0D79771E
:105FB100126DB5E49000D1F0227BFF7A0D79971232
:0C5FC1006DB57578029000D17409F022D3
:1055FC009000CEE0FF127142400302568A9000CE1A
:10560C00E0FF90003CE0FE04F074032EF582E434DD
:10561C0000F583EFF090003CE0D3940540729000CD
:10562C0004E0540F75F00AA4FFA3E0540F2F90036D
:10563C00F2F09003F5F0900007E0540F75F00AA417
:10564C00FF900006E0540F75F064A42FFF90000843
:10565C00E0540F2F9003F3F0C22FC20EC22DC20BD9
:10566C00C230C20D7880760812573AD231D20F7BF5
:10567C00FF7A0D7987126DB5E49000D1F0227BFF93
:10568C007A0D7997126DB57578029000D17409F086
:01569C0022EB
:0D715100E578700812368AE49000D1F02233
:1070F0007516027517ABD230D20D7BFF7A0D79A7CA
:03710000026DE637
:106737009003FAE0B40A005043906747F82828739B
:1067470002676502676802676B02676E026771021C
:10675700677402677702677A02677D026780027053
:10676700150270DC025DA502634A026107026CDE56
:0D6777000257D302596702555812715E2275
:107015009000CDE0FFB42A079003FAE004F022EFD8
:0A702500B423069003FA7405F0226C
:1070DC009000CDE0B42A079003FAE004F022E4908B
:0470EC0003FAF02291
:105DA5009000CDE0B4310D7BFF7A0D7917126DB5FA
:105DB500B244802C9000CDE0B432107BFF7A0D798F
:105DC50027126DB5B24312573A80159000CDE0B455
:105DD50033187BFF7A0D7937126DB5B25812573AE1
:105DE5007578029003FA7409F0229000CDE0FFB4B3
:105DF500340D90003C740AF09003FAE004F022EFB1
:105E0500B4350C90003C740AF09003FA7404F02247
:10634A009000CDE0FF127142504B9000CDE0FF90DB
:10635A00003CE0FE04F074032EF582E43400F58379
:10636A00EFF090003CE0D3940B402F7BFF7A0D793D
:10637A0047126DB590000DE0540F75F00AA4FFA303
:10638A00E0540F2F9003F4F012573A7578029003F5
:0B639A00FA7409F022E49003FAF022EC
:106107009000CDE0FF12714250589000CDE0FF9013
:10611700003CE0FE04F074032EF582E43400F583BE
:10612700EFF090003CE0D3940C403C7BFF7A0D7974
:1061370057126DB590000EE0540F75F00AA4FF904A
:10614700000DE0540F75F064A42FFF90000FE0548A
:106157000F2FF533F532F52F7578029003FA74098E
:08616700F022E49003FAF0229B
:106CDE009000CDE0FFB4310D90003C7401F09003B4
:106CEE00FAE004F022EFB4320D90003C7401F09003
:106CFE0003FA7407F022EFB4330C90003C7401F0E9
:076D0E009003FA7408F02263
:1057D3009000CDE0FF127142506C9000CDE0FF903D
:1057E300003CE0FE04F074032EF582E43400F583FC
:1057F300EFF090003CE0D39403405D1262365046D4
:10580300C22FC231C20EC20F900036E0FF25E02442
:1058130091F582E4340CF583E493F516740193F562
:1058230017EF75F010A42451F9740235F0FA7BFFD9
:10583300126DE6D230D20D7BFF7A0D7967126DB50A
:10584300E49003FAF0227BFF7A0D7997126DB57518
:0958530078029003FA7409F022B6
:105967009000CDE0FF12714250649000CDE0FF90AF
:10597700003CE0FE04F074032EF582E43400F58366
:10598700EFF090003CE0D3940340551261D6503EAF
:10599700C20FC231C22DC20BC230C20D7887760842
:1059A700900037E0FF121237D20E7BFF7A0D79771E
:1059B700126DB5900037E075F010A42491F97405C5
:1059C70035F0FA7BFF126DE6E49003FAF0227BFFD5
:1059D7007A0D7997126DB57578029003FA7409F00C
:0159E700229D
:105558009000CDE0FF12714240030255E99000CD62
:10556800E0FF90003CE0FE04F074032EF582E43482
:1055780000F583EFF090003CE0D39405407590006F
:1055880004E0540F75F00AA4FFA3E0540F2F900312
:10559800F2F09003F5F0900007E0540F75F00AA4BC
:1055A800FF900006E0540F75F064A42FFF900008E8
:1055B800E0540F2F9003F3F0C22FC20EC22DC20B7E
:1055C800C230C20D7880760812573AD231D20F7B9A
:1055D800FF7A0D7987126DB51244DFE49003FAF073
:1055E800227BFF7A0D7997126DB57578029003FAD0
:0455F8007409F02220
:0D715E00E578700812368AE49003FAF022FA
:10402900003800512372461765340E5F2D7C4819FC
:104039006B3A1C4D3F6E5A0B792812433160540577
:104049007726001F3D227A654758756A48570F1031
:10405900322D6877554A120D2F301D02203F67789F
:104069005A45006245270B694E2C157750321E7C44
:104079005B39294B6C0E224067053C5E791B37552D
:10408900721052301775593B1C7E472502604C2E21
:10409900096B7B193E5C701235576E0C2B4965070D
:1040A9002042264463012D4F680A33517614385A49
:1040B9007D1F0F6D4A28046641231A785F3D1173ED
:1040C9005436741631537F1D3A58610324466A08E1
:1040D9002F4D5D3F187A56341371482A0D6F4321CD
:1040E90006644F2D0A68442601635A381F7D5133EF
:1040F9001476660423416D0F284A73113654781AD1
:104109003D5F1D7F583A16745331086A4D2F03617C
:104119004624345671133F5D7A18214364062A48B0
:104129006F0D690B2C4E620027457C1E395B771594
:104139003250402205674B290E6C553710725E3C90
:104149001B793B597E1C305275172E4C6B0925473C
:10415900600212705735197B5C3E076542200C6E70
:10416900492B004307440D4E0A49195A1E5D14573D
:104179001350317236753C7F3B78286B2F6C25665E
:024189002261B1
:10573A00788676ACA258E433FFC4333354C0FE9063
:10574A0003F4E0FD541F25E04EFE9003F2E0FC5402
:10575A0010C4540F4E7885F6EC540FC454F0FE90E2
:10576A0003F3E0FC54F0C4540F4E7884F6EC540F63
:10577A00C454F0FE9003F5E0FC541EC3134E788324
:10578A00F6EF3395E0FE74292FF58274403EF583D7
:10579A00E493FFED90402B93FEEF6EFF9003F2E04F
:1057AA0090404B936FFF9003F3E090406B936FFF31
:1057BA00EC90416B936F7882F69003F5E030E00449
:0957CA00E64480F678817628227D
:0300000002718FFB
:0C718F00787FE4F6D8FD758196025192DD
:10525E00BB010CE58229F582E5833AF583E0225005
:10526E0006E92582F8E622BBFE06E92582F8E2224F
:0D527E00E58229F582E5833AF583E4932269
:10528B00BC000BBE0029EF8DF084FFADF022E4CC07
:10529B00F875F008EF2FFFEE33FEEC33FCEE9DECD0
:1052AB00984005FCEE9DFE0FD5F0E9E4CEFD22ED16
:1052BB00F8F5F0EE8420D21CFEADF075F008EF2F60
:1052CB00FFED33FD4007985006D5F0F222C398FD51
:0552DB000FD5F0EA22EE
:1052E000A3F8E0C5F025F0F0E58215827002158381
:0652F000E0C838F0E822DE
:0C52F600A42582F582E5F03583F58322C3
:10530200D083D082F8E4937012740193700DA3A33A
:1053120093F8740193F5828883E47374029368604E
:06532200EFA3A3A380DF4E
:00000001FF
